:100000000C94E0070C9408080C9408080C94080859
:100010000C9408080C9408080C9408080C94080820
:100020000C9408080C9408080C94951A0C94041B62
:100030000C9408080C9408080C9408080C94080800
:100040000C9408080C9408080C9408080C940808F0
:100050000C9408080C9408080C9408080C94361D9D
:100060000C9408080C9408080C9408080C940808D0
:100070000C9408080C9408080C9408080C940808C0
:100080000C9408080C9408080C9408080C940808B0
:100090000C9408080C9408080C9408080C940808A0
:1000A0000C9408080C9408080C9408084461790022
:1000B00041636374004C6F616E00436170616369FA
:1000C0007479200053707261792000050512151FA4
:1000D000150905082466E766244120596573202028
:1000E00042204E6F000043616E6479204361737457
:1000F0006C6500536F6461205377616D70004775C4
:100100006D6D7920466F726573740043686F636F1D
:100110006C616E640049636520437265616D2052B5
:1001200064005377656574205375697465730000C6
:100130004C6F6C6C7900536F757273004D61727304
:10014000004165726F004865727368657900502ED2
:100150005375676172002000200003081F051F1FF0
:10016000151B1F11111F110E1F15111F05011F1146
:100170001D1F041F001F0010101F1F041B1F101045
:100180001F061F1F011F1F111F1F05071F311F1FE4
:10019000051B17151D011F011F101F0F100F1F0C2E
:1001A0001F1B041B071C071915130C121E1F120C12
:1001B0001E12120C121F0C1A14041F052E2A1E1FC9
:1001C000021C001D00201D001F041A011F001E0438
:1001D0001E1E021E1E121E3E120C0C123E1E020697
:1001E00014120A020F121E101E0E100E1E081E1AE6
:1001F000041A2E281E1A12161F111F001F001D158B
:100200001711151F07041F17151D1F151D01011FAD
:100210001F151F17151F00170000100020100000E9
:10022000030004083E09093E3F25251A1E2121121C
:100230003F21211E3F2525213F0505011E21293A89
:100240003F04043F213F21001021211F3F040A31B8
:100250003F2020203F02023F3F02043F1E21211E7B
:100260003F0909061E21112E3F09093622252519AD
:10027000013F01011F20201F0F10201F3F10103FC2
:100280003B04043B03043807312D2321102A2A3C68
:100290003F2424181C2222141824243F1C2A2A2C10
:1002A000047E05014C52523E3F040438243D200098
:1002B0004040443D3F081422213F20003E04043EBC
:1002C0003E04023C1C22221C7E22221C1C22227E76
:1002D0003E040204242A2A12021F22201E20201E6D
:1002E0000E10201E3E10103E360808364E50503E6E
:1002F000322A26221E29251E223F200032292926A5
:100300001221251A0C0A3F08172525191E25251824
:10031000013905031A25251A0629291E002F000078
:10032000002000004020000000030000000000004A
:10033000003E5B4F5B3E3E6B4F6B3E1C3E7C3E1C6B
:10034000183C7E3C181C577D571C1C5E7F5E1C00B1
:10035000183C1800FFE7C3E7FF0018241800FFE768
:10036000DBE7FF30483A060E2629792926407F052B
:100370000507407F05253F5A3CE73C5A7F3E1C1C41
:1003800008081C1C3E7F14227F22145F5F005F5F01
:1003900006097F017F006689956A606060606094ED
:1003A000A2FFA29408047E040810207E20100808F2
:1003B0002A1C08081C2A08081E101010100C1E0CFD
:1003C0001E0C30383E3830060E3E0E06000000008F
:1003D0000000005F00000007000700147F147F1476
:1003E000242A7F2A122313086462364956205000BB
:1003F00008070300001C2241000041221C002A1CA7
:100400007F1C2A08083E0808008070300008080891
:100410000808000060600020100804023E514945B1
:100420003E00427F400072494949462141494D33CF
:100430001814127F1027454545393C4A4949314136
:10044000211109073649494936464949291E000004
:100450001400000040340000000814224114141459
:100460001414004122140802015909063E415D5945
:100470004E7C1211127C7F494949363E414141224E
:100480007F4141413E7F494949417F090909013E78
:10049000414151737F0808087F00417F410020409F
:1004A000413F017F081422417F404040407F021CB1
:1004B000027F7F0408107F3E4141413E7F090909C8
:1004C000063E4151215E7F09192946264949493294
:1004D00003017F01033F4040403F1F2040201F3F5A
:1004E0004038403F631408146303047804036159DF
:1004F000494D43007F414141020408102000414121
:10050000417F0402010204404040404000030708CC
:100510000020545478407F284444383844444428C8
:10052000384444287F385454541800087E0902186F
:10053000A4A49C787F0804047800447D40002040F7
:10054000403D007F1028440000417F40007C04783B
:1005500004787C080404783844444438FC18242483
:100560001818242418FC7C08040408485454542403
:1005700004043F44243C4040207C1C2040201C3C80
:100580004030403C44281028444C9090907C446477
:10059000544C44000836410000007700000041360A
:1005A000080002010204023C2623263C1EA1A16190
:1005B000123A4040207A38545455592155557941C2
:1005C0002154547841215554784020545579400C99
:1005D0001E5272123955555559395454545939557A
:1005E0005454580000457C410002457D42000145BD
:1005F0007C40F0292429F0F0282528F07C5455452A
:10060000002054547C547C0A097F493249494932BC
:100610003248484832324A4848303A4141217A3AD1
:1006200042402078009DA0A07D39444444393D409B
:1006300040403D3C24FF2424487E4943662B2FFC48
:100640002F2BFF0929F620C0887E090320545479F6
:10065000410000447D413048484A32384040227AC7
:10066000007A0A0A727D0D19317D2629292F282644
:100670002929292630484D4020380808080808084C
:100680000808382F10C8ACBA2F102834FA00007BA5
:10069000000008142A142222142A140895002200AB
:1006A00095AA005500AAAA55AA55AA000000FF0065
:1006B000101010FF00141414FF001010FF00FF10A2
:1006C00010F010F0141414FC001414F700FF0000D4
:1006D000FF00FF1414F404FC141417101F10101F53
:1006E000101F1414141F00101010F0000000001F41
:1006F000101010101F10101010F010000000FF104C
:100700001010101010101010FF10000000FF140047
:1007100000FF00FF00001F10170000FC04F4141479
:100720001710171414F404F40000FF00F714141445
:1007300014141414F700F7141414171410101F10C5
:100740001F141414F4141010F010F000001F101FE8
:100750000000001F14000000FC140000F010F01056
:1007600010FF10FF141414FF141010101F000000CD
:1007700000F010FFFFFFFFFFF0F0F0F0F0FFFFFFD1
:100780000000000000FFFF0F0F0F0F0F3844443828
:10079000447C2A2A3E147E02020606027E027E0263
:1007A00063554941633844443C04407E201E200682
:1007B000027E020299A5E7A5991C2A492A1C4C72BF
:1007C00001724C304A4D4D303048784830BC625A46
:1007D000463D3E494949007E0101017E2A2A2A2AD6
:1007E0002A44445F444440514A444040444A5140B2
:1007F0000000FF0103E080FF000008086B6B083673
:1008000012362436060F090F0600001818000000E3
:100810001010003040FF0101001F01011E00191DD2
:100820001712003C3C3C3C0000000000D5F08D1449
:10083000A1C881CFD9F1AF20005810F0F89C8E8765
:1008400083878E9CF8F00000FEFF03030303030779
:100850000EFCF80000FEFF0303030303070EFCF881
:100860000000FFFF00000000000000FFFF0000FE8E
:10087000FF8383838383C7EE7C380000F8FC0E0778
:10088000030303070EFCF800003F7FE0C08080C038
:10089000E07F3FFFFF01010101010101FFFF0000B7
:1008A000FFFF0C0C0C0C1C3E77E3C100007FFFC067
:1008B000C0C0C0C0E0703F1F00001F3F70E0C0C05C
:1008C000C0E0703F1F00007FFFC1C1C1C1C1E3771D
:1008D0003E1C00001F3F70E0C0C0C0E0703F1F0022
:1008E0000000000001FFFF01000000647572696EE6
:1008F00067207468652063686173652121006275F3
:10090000636B732066726F6D207075727365730010
:10091000596F7520736E6174636865642000546854
:10092000657920616C6C20676176652075702100A7
:1009300041204D6F6D206761766520757021210023
:10094000002020596F75206D697373656421212122
:1009500000006861766520746F2072756E210061F9
:100960006E792073707261792120596F7500596F0B
:100970007520646F6E277420686176650074686501
:100980006D2100596F752063616E27742073686153
:100990006B6500616E20616C6C6579212100596F77
:1009A00075206C6F7374207468656D20696E0075B6
:1009B0006E697473206F663A2000596F7520666FF8
:1009C000756E642000323030206275636B733F00B7
:1009D0006D6F726520737061636520666F7200636E
:1009E000616E6479207361636B2077697468005766
:1009F000696C6C20796F75206275792061206E6555
:100A0000770057696C6C20796F7520656174206977
:100A1000743F006D6F73746C7920756E63686577D1
:100A20006564212100686572652074686174206CBA
:100A30006F6F6B73005468657265277320736F6DF9
:100A4000652067756D00646F6C6C6172733F007335
:100A50007072617920666F7220343030004D6F6D96
:100A600020726570656C6C616E74007374696E6B76
:100A700020737072617920666F7200736C656570A7
:100A800020737072617920666F7200343030206498
:100A90006F6C6C6172733F0057696C6C20796F7575
:100AA00020627579206100616674657220796F75C6
:100AB0002100667269656E64732061726500206F43
:100AC000662068657200616E642000596F7572203F
:100AD0004D6F7468657200746F2063686172697429
:100AE000792100596F752067617665206120626900
:100AF0007400617265206F7574726167656F7573DC
:100B0000212121210073686F727461676521205073
:100B1000726963657300506F7764657265642073F2
:100B200075676172007072696365732121210061CC
:100B300074206F7574726167656F75730062757983
:100B4000696E6720486572736865790043686F63F2
:100B50006F686F6C696373206172650062616B65B9
:100B60002D6F6666212121210066726F6D206C61F8
:100B70007374207765656B27730063686561702007
:100B800048657273686579004D6F6D732061726599
:100B90002073656C6C696E6700626F74746F6D654D
:100BA00064206F7574212121004D61727320707271
:100BB000696365732068617665006C6F6C6C792180
:100BC0002121006172652073656C6C696E6720631A
:100BD00068656170004B6964732061742073636899
:100BE0006F6F6C00746F6461792100626F72726F55
:100BF000776564206D6F6E657900596F7520616C43
:100C00007265616479002100596F7520646F6E27E9
:100C100074206861766520616E7900004F6F707393
:100C200021002100596F752063616E277420616671
:100C3000666F726400004F6F7073210021006D6F4A
:100C400072652000596F752063616E27742063619F
:100C500072727900004F6F70732100457874656E71
:100C60006465642047616D653A00004E6F726D6186
:100C70006C2047616D653A00596F75277265206376
:100C800061756768742121006265656E206869740A
:100C90002100596F75277665006D6973736564214E
:100CA00021005468657900796F752121200054680E
:100CB0006579277265206E616767696E67004120FC
:100CC00053707261792020422052756E0045525255
:100CD0004F522000004F6C64200048696768205321
:100CE000636F72653A000047616D65206F766572CB
:100CF000212053636F72653A00416D740053617631
:100D0000696E677300596F75206F776500596F754D
:100D10002068617665005769746864726177204D58
:100D20006F6E6579004465706F736974204D6F6EE6
:100D3000657900426F72726F77204D6F6E65790032
:100D4000506179204C6F616E000000517479005041
:100D50007269636500436F73747300596F7520681F
:100D60006176650053656C6C200042757920000047
:100D700000796F75722074656574683F0064656EF4
:100D80007469737420746F2066697800646F6C6C8A
:100D900061727320666F7220610057696C6C2079F4
:100DA0006F7520706179203130303000596F757265
:100DB000206865616C74683A20007374696C6C20FB
:100DC000616674657220796F752100204D6F6D73B7
:100DD0000054686572652061726520004265696E25
:100DE00067206368617365642121005769746864D2
:100DF000726177204D6F6E6579004465706F73691D
:100E000074204D6F6E65790042616E6B00426F72A7
:100E1000726F77204D6F6E65790052657061792031
:100E20004C6F616E0052696368204275646479009A
:100E30004A65742066726F6D200053656C6C2043A8
:100E4000616E6479004275792043616E6479004374
:100E5000616E6479205361636B0042616E6B005276
:100E6000696368204275646479004A65740043616F
:100E70006E6479205361636B0053656C6C20436131
:100E80006E6479004275792043616E647900486927
:100E900067682053636F72657300457874656E648C
:100EA00065642047616D6500486974207468652039
:100EB0005377656574730076312E322E30004361AE
:100EC0006E6479576172001E1E0000000000000071
:100ED000000000000000C0F0E8C48202033F3F0FA2
:100EE0008782C2C4C8F0C0000000000000008080FB
:100EF000807088A80FF1810181C1E1F0FCF00081D0
:100F00008143271F0700000000008040A1562C14D9
:100F100034224176080D090701010101010000009A
:100F20000000003028140A05020100000000000043
:100F300000000000000000000000000000000000B1
:100F400000080B0002020200000904000001020276
:100F500000000524001001052401010104240206FB
:100F60000524060001070581031000400904010063
:100F7000020A000000070502024000000705830284
:100F80004000000403090412010002EF0201404185
:100F900023368000010102030141726475696E6F9E
:100FA000204C4C430041726475696E6F204C656F34
:100FB0006E6172646F0003051F0E0400B31D813063
:100FC00011241FBECFEFDAE0DEBFCDBF12E0A0E0FC
:100FD000B1E0EAE3FEE602C005900D92A234B1074B
:100FE000D9F727E0A2E4B2E001C01D92A438B2070D
:100FF000E1F717E0CFEDD7E004C02197FE010E9492
:101000000F35CE3DD107C9F70E94341E0C9410371E
:101010000C940000E6EDF2E0A0E0B8E000800EBC29
:101020008111012C1197A0FDFDCF0192B9F70DB4EC
:101030000895480F592F511D1416150684F5803850
:1010400091056CF597FF02C090E080E041385105B2
:1010500014F040E850E0481BFB01E770FF2721E057
:1010600001C0220FEA95EAF777FF02C0695F7F4F60
:10107000FB0133E0F595E7953A95E1F7F695FE2FFC
:10108000EE27F795E795E80FF91FEA52FD4F41501B
:1010900030F08191DF011197822B8C93F8CF089566
:1010A0006F927F928F929F92AF92BF92CF92DF9278
:1010B000EF92FF920F931F93CF93DF93DC017A019E
:1010C0004115510509F49CC0FA01149131965491CF
:1010D000F2E0EF0EF11CC12FD0E0222309F1CC2465
:1010E000C394D12C852F877011F4D12CC12CE52FFE
:1010F000E695E695E695EC0DFD2DF11DEC9FC00102
:10110000ED9F900DFC9F900D1124033011F4880F7A
:10111000991F289FF001299FF00D1124EE0EFF1E4C
:10112000FD01EC0FFD1F1E161F060CF069C0A03854
:10113000B1050CF065C0CB01850F911D181619067D
:101140000CF05EC0603471050CF05AC0E114F1047B
:1011500009F456C0362F3770CB0177FD079623E090
:10116000959587952A95E1F7282F77FF04C03323BB
:1011700011F02FEF280F662777276A1B7B0BB7FD2F
:1011800002C070E060E090E89A1BE038F1050CF4D2
:10119000912F961BE22F022E000CFF0BDE2ED09417
:1011A0002F3F0CF0D12C41E0852F877009F440E0EF
:1011B000B52EB694B694B6944B0DE40FF11D399745
:1011C00014F048E0421BB42EBD182D0D40E8240356
:1011D000F0011124AE0FBF1FA60FB71F1D9D600D9C
:1011E000711D1124A701460F571FC32E032E000C9B
:1011F000DD08033009F4C7C090F4023009F474C06C
:10120000DF91CF911F910F91FF90EF90DF90CF90E2
:10121000BF90AF909F908F907F906F9008950A3FFE
:10122000A1F1B20E0B3F61F72B1551F3BD016A52CC
:101230007D4F10E000E0091708F09FC0FA01E00FB1
:10124000F11FE491F0E04F010C2C02C0880C991CB6
:101250000A94E2F727FD06C0FB018081F82CF09488
:101260008F218083332361F0273054F47B01F0E831
:10127000EF0EF11CA92CA094F70180818A218083B4
:101280000F5F1F4F6F5F7F4FD6CFB20E2B1509F444
:10129000B7CFBD016A527D4F10E000E0091708F09A
:1012A00066C0FA01E00FF11FE491F0E04F010C2C51
:1012B00002C0880C991C0A94E2F727FD04C0FB01C8
:1012C000808188298083332351F0273044F47B01C7
:1012D000F0E8EF0EF11CF7018081892980830F5F10
:1012E0001F4F6F5F7F4FDACF6FEF70E0032E02C0AA
:1012F000660F771F0A94E2F760957095972E8B2CF6
:10130000820E281509F47CCF8D010A521D4FF12C55
:10131000E12CE91630F5FA01EE0DFF1DE491F0E045
:101320003F010C2C02C0660C771C0A94E2F727FDE3
:1013300005C0F8018081862386298083332359F0F4
:1013400027304CF45801F0E8AF0EB11CF501808154
:10135000892187298083FFEFEF1AFF0A0F5F1F4F54
:10136000D8CF2F5F4C0F5D1FA058BF4FCACF2F5F44
:101370004C0F5D1FA058BF4F89CF2F5F4C0F5D1FD3
:10138000A058BF4F51CFE92EF12CFA01E60FF71FFD
:10139000AA52BD4F60E870E06E197F09CE19DF09CF
:1013A0008E01000F111F41E050E07A01032E01C0B1
:1013B000EE0C0A94EAF7592F4B2D892E932ECF93DA
:1013C000DF93ED01EF96EF962296A590C5909920B8
:1013D00059F0AE9C5001CE9C600127302CF4F8806F
:1013E000D094FD20FB28F99222233AF0FC90C0947F
:1013F000FC20FA28FD920C94FE0911965A9529F7C3
:101400004A9551F0582D23951124E00FF11DA60F98
:10141000B11DC60FD11DD9CFDF91CF911124F0CED0
:101420000F9302E020E00E9450080F9108952F9240
:101430003F924F925F926F927F928F929F92AF9264
:10144000BF92CF92DF92EF92FF920F931F93CF93B1
:10145000DF93CDB7DEB728970FB6F894DEBF0FBE87
:10146000CDBF6F836A0119011C830B83FE82ED825D
:10147000811128C005E010E029E030E03A8329839B
:10148000B6010D2C000C880B990B0E94C0314B014A
:101490005C015F8151111DC0E4E4F7E090E080E061
:1014A00018861F828C159D050CF02BC12481358177
:1014B0004F8158854217530714F438872F830196BC
:1014C0003696F0CF04E010E048E050E05A834983BC
:1014D000D7CF20E030E040E05FE30E941F324B01B5
:1014E0005C0120E030E0A9010E94FA3420E030E005
:1014F00040E05FE387FD30C0C501B4010E948E3338
:101500000E946C3478876F83A6018F819885481B71
:10151000590BE4E4F7E090E080E0B12CA12C2F819E
:10152000388582179307ECF086E0829FF001839F55
:10153000F00D1124EC5BF84F90E080E0D12CC12C31
:1015400084179507BCF424813581C216D3060CF4A8
:10155000690101963696F4CFC501B4010E948D331E
:10156000CFCF24813581A216B3060CF45901019620
:101570003696D5CFB801110F880B990B0E94C03158
:101580002B013C01B5016C0D7D1D072E000C880B55
:10159000990B0E94C03120E030E040EE5FE30E94F2
:1015A0008E336B017C0120E030E040E05FE3C3015B
:1015B000B2010E941F329B01AC01C701B6010E941B
:1015C0001F326B017C0120E030E0A9010E94FA3457
:1015D00020E030E040E05FE387FD89C0C701B6014D
:1015E0000E948E330E946C3402E410E0061B170B3D
:1015F000F10111830083B501BB0C880B990B0E948C
:10160000C03120E030E040EE5FE30E948E33A30162
:1016100092010E941F324B015C0120E030E0A901E1
:101620000E94FA3420E030E040E05FE387FD64C0D0
:10163000C501B4010E948E330E946C34600F711F8B
:10164000EB81FC817183608329813A81B901330F79
:10165000880B990B0E94C03120E030E040E05FE34E
:101660000E941F326B017C014F815885BA01550FD2
:10167000880B990B0E94C0319B01AC01C701B601D8
:101680000E941F326B017C0120E030E0A9010E9422
:10169000FA3420E030E040E05FE387FD85C0C70119
:1016A000B6010E948E330E946C342AE230E0C901F8
:1016B000861B970BED81FE819183808328960FB660
:1016C000F894DEBF0FBECDBFDF91CF911F910F9178
:1016D000FF90EF90DF90CF90BF90AF909F908F9052
:1016E0007F906F905F904F903F902F900895C7012B
:1016F000B6010E948D3376CFC501B4010E948D33AF
:101700009BCFB801110F880B990B0E94C03120E0CC
:1017100030E040E05FE30E941F322B013C01EF818B
:10172000F885BF01FF0F880B990B0E94C0319B0108
:10173000AC01C301B2010E941F322B013C0120E029
:1017400030E0A9010E94FA3420E030E040E05FE39D
:1017500087FD25C0C301B2010E948E330E946C3404
:1017600022E430E0C901861B970BF101918380834D
:101770008FEF9FEFEB81FC819183808329813A81F8
:10178000B901330F880B990B0E94C03120E030E083
:1017900040E05FE30E941F32A501940171CFC301B5
:1017A000B2010E948D33DACFC701B6010E948D339A
:1017B0007ACFFC018091D502882311F13FB7F894CC
:1017C00082E08093E9002091F200822F90E01816C9
:1017D000190614F481E090E0882339F0289844E653
:1017E0004093D4024091F1004083222339F02091AC
:1017F000F200211103C02BE62093E8003FBF0895BB
:101800008FEF9FEF08952FB7F89483E08093E9005E
:101810009091E800892F807295FF04C09091F200AA
:1018200080E4891B2FBF08958091CC0281110DC0E7
:1018300082E08093C80284E08093C9021092CB02B8
:101840001092CA0281E08093CC0288EC92E0089565
:10185000CF93DF931F92CDB7DEB76983DC01ED91A3
:10186000FC910280F381E02D41E050E0BE016F5F0A
:101870007F4F09950F90DF91CF91089583E080937A
:10188000E9008091F200882319F08AE38093E80050
:1018900008950E94030C90E00895CF93DF931F9268
:1018A000CDB7DEB7FC018485958597FD08C02FEF85
:1018B0003FEF358724870F90DF91CF910895CE01B8
:1018C00001960E94D90B019719F4898190E0F3CF1A
:1018D0008FEF9FEFF0CF0F931F93CF93DF931F9264
:1018E000CDB7DEB78C01FC018485958597FF0BC0D1
:1018F000CE0101960E94D90B019771F4898190E085
:10190000F80195878487F801848595850F90DF918C
:10191000CF911F910F9108958FEF9FEFF1CFFC01B1
:101920008485958597FD0BC09FB7F89482E08093DE
:10193000E9008091F2009FBF90E0019608959FB763
:10194000F89482E08093E9008091F2009FBF90E0DC
:1019500008954091C2025091C3022091C00230917B
:10196000C10242175307B4F49091E8009570E1F377
:101970009091E80092FD19C08093F1008091C2021D
:101980009091C30201968F739927892B19F48EEFDA
:101990008093E8008091C2029091C30201969093D7
:1019A000C3028093C20281E0089580E00895DF922F
:1019B000EF92FF920F931F93CF93DF93D82E8A015C
:1019C000EB017B01E40EF51ECE15DF0559F0D7FEC5
:1019D00012C0FE0184910E94A90C21968111F4CFBE
:1019E0000FEF1FEFC801DF91CF911F910F91FF9073
:1019F000EF90DF9008958881EECF0F931F93CF93E0
:101A0000DF931F92CDB7DEB782E0898342E450E0D6
:101A100061E47FE080E80E94D70C0E94140CDC0196
:101A200012960D911C910115110589F0D801ED91C7
:101A3000FC910280F381E02DBE016F5F7F4FC801F2
:101A4000099597FD04C0F80100851185ECCF8981C7
:101A50000F90DF91CF911F910F910895615030F059
:101A60002091F100FC0120830196F8CF289884E6AC
:101A70008093D40208953FB7F8948091BC0290916E
:101A8000BD02A091BE02B091BF0226B5A89B05C0C1
:101A90002F3F19F00196A11DB11D3FBFBA2FA92FED
:101AA000982F8827BC01CD01620F711D811D911DEA
:101AB00042E0660F771F881F991F4A95D1F7089556
:101AC0008F929F92AF92BF92CF92DF92EF92FF924E
:101AD0006B017C010E943B0D4B015C01C114D104E0
:101AE000E104F104B9F00E943B0D681979098A09F3
:101AF0009B09683E73408105910580F321E0C21A7D
:101B0000D108E108F10888EE880E83E0981EA11C38
:101B1000B11CE4CFFF90EF90DF90CF90BF90AF90DB
:101B20009F908F9008958F929F92AF92BF92CF9285
:101B3000DF92EF92FF920F931F93CF93DF936C018D
:101B40007B018A0180911401882309F45CC0809193
:101B5000D502882309F457C08091C70280FF05C0D1
:101B60008091E00082608093E000E801B12C8AEF70
:101B7000A82E93E0892E2AE3922E209711F4BB2001
:101B8000D9F10E94030C81110AC0AA94AA20D9F1AC
:101B900061E070E080E090E00E94600DEECF8C1775
:101BA0001D0611F00CF08C2F9FB7F8948092E9007D
:101BB0002091E80025FD02C09FBFDFCF282F30E035
:101BC000C21BD30BF701815020F041914093F100EB
:101BD000FACFE20EF31EBB2021F09092E800B12C68
:101BE000EBCF8091E80085FDE7CF9092E800BB2421
:101BF000B394209709F3F3CF5D9884E68093C602EF
:101C0000101611063CF081E090E0F6019383828388
:101C100010E000E0C801DF91CF911F910F91FF907C
:101C2000EF90DF90CF90BF90AF909F908F900895EE
:101C30000895DB0114964D915C9115976D917C91FF
:101C4000DC01ED91FC910280F381E02D09942F924B
:101C50003F924F925F926F927F928F929F92AF923C
:101C6000BF92CF92DF92EF92FF920F931F93CF9389
:101C7000DF9300D000D000D0CDB7DEB7782E662E2F
:101C80005A0128E0422E512C811103C099E0492EBF
:101C9000512CCE0101967C018E010D5F1F4F9E01DC
:101CA0002B5F3F4FA501662D872D0E94170AB501B6
:101CB0000B2C000C880B990B0E94C03120E030E007
:101CC00040E05FE30E941F326B017C0120E030E0C6
:101CD000A9010E94FA3420E030E040E05FE387FD94
:101CE00024C0C701B6010E948E330E946C348B0160
:101CF00084E4C82E87E0D82E049D1001059D300C89
:101D0000149D300C1124F12CE12C912C812C8A147F
:101D10009B04B4F589819A81662019F0801691069A
:101D20004CF42D818E0D9F1D0BC0C701B6010E9482
:101D30008D33DBCF2B81A70142195309840F951FE7
:101D40007720A1F020936D0720936C0780936E0796
:101D5000B60188E697E00E94190E9FEF891A990A4A
:101D600086E0C80ED11CE40CF51CD1CF2093770778
:101D70002093760780937807B60182E797E0EBCF50
:101D800026960FB6F894DEBF0FBECDBFDF91CF9180
:101D90001F910F91FF90EF90DF90CF90BF90AF9089
:101DA0009F908F907F906F905F904F903F902F907B
:101DB0000895EF92FF920F931F93CF93DF938C01BF
:101DC0007B01D0E0C0E0F701EC0FFD1F64916623BA
:101DD00061F0D801ED91FC910190F081E02DC801F6
:101DE0000995892B11F02196EECFCE01DF91CF918D
:101DF0001F910F91FF90EF900895AF92BF92CF92F5
:101E0000DF92EF92FF920F931F93CF93DF936C01BA
:101E10007B018B01040F151FEB015E01AE18BF089B
:101E2000C017D10759F06991D601ED91FC9101904D
:101E3000F081E02DC6010995892B79F7C501DF9165
:101E4000CF911F910F91FF90EF90DF90CF90BF90B7
:101E5000AF900895BC0190E080E00C94600D8FB1CC
:101E60008095807F669B88601C9B8460089590911C
:101E70004A02982329F490914B02982381E009F4B7
:101E800080E0089580389105B8F460347105A0F4BD
:101E900020E191E061FD94E060FD990F62FD929573
:101EA000687F269FD0011124A80FAA52BD4F8C91A4
:101EB00040FF03C0892B8C93089590958923FBCF15
:101EC0002F923F924F925F926F927F928F929F924A
:101ED000AF92BF92CF92DF92EF92FF920F931F9338
:101EE000CF93DF937C016B0188248394912CD0E005
:101EF000C0E005E010E096EF692E77247A942CEF8D
:101F0000A22EBB24BA94842F8470582E842F827002
:101F1000482E842F8870382E4170242E219682E01E
:101F2000880E911CA80CB91C552091F041E0B80115
:101F30006C0D7D1DC7018C0F9D1F0E94420F41E05B
:101F4000B6016C0F7D1FC8018E0D9F1D0E94420FB0
:101F5000442091F041E0B601601B710BC7018C0F6A
:101F60009D1F0E94420F41E0B6016C1B7D0BC80112
:101F70008E0D9F1D0E94420F332091F041E0B6016B
:101F80006C0F7D1FC701801B910B0E94420F41E027
:101F9000B8016C0D7D1DC7018C1B9D0B0E94420F6B
:101FA000222091F041E0B6016C1B7D0BC701801B24
:101FB000910B0E94420F41E0B601601B710BC701FB
:101FC0008C1B9D0B0E94420FC017D10754F4B7FC25
:101FD000A5CF0150110982E0680E711CA60CB71C38
:101FE0009DCFDF91CF911F910F91FF90EF90DF90E8
:101FF000CF90BF90AF909F908F907F906F905F90A9
:102000004F903F902F9008952F923F924F925F9262
:102010006F927F928F929F92AF92BF92CF92DF92F8
:10202000EF92FF920F931F93CF93DF93EC0141E068
:102030006FE370E00E94420F41E065E370E0CE0183
:102040000E94420F41E06AE370E0CE0105960E94D3
:10205000420F41E06AE370E0CE0105970E94420F13
:1020600022242394312CF12CE12C05E010E036EFF2
:10207000432E55245A944CEFC42EDD24DA948FEF6E
:10208000E81AF80A82E0280E311CC20CD31C470162
:102090008C0E9D1E41E058018AE3A80EB11CB501CB
:1020A000C4010E94420F3E016E187F0841E0B50155
:1020B000C3010E94420F41E08AE3A82EB12CA01A6E
:1020C000B10AB501C4010E94420F41E0B501C3014C
:1020D0000E94420F47018AE3880E911C41E0B4013F
:1020E0005E01A00EB11EC5010E94420F41E0B40185
:1020F0003E01601A710AC3010E94420F9AE3892EC1
:10210000912C8E189F0841E0B401C5010E94420F36
:1021100041E0B401C3010E94420FE016F1069CF0B9
:10212000DF91CF911F910F91FF90EF90DF90CF90B3
:10213000BF90AF909F908F907F906F905F904F90E7
:102140003F902F900895D7FC9ACF0150110982E05B
:10215000480E511CC40CD51C92CF8F929F92AF9207
:10216000BF92CF92DF92EF92FF920F931F93CF9384
:10217000DF936D3089F0C0904802D09049026A30F8
:10218000D1F4109247021092460288E0C80ED11C8A
:10219000D0924902C092480281E090E0DF91CF9155
:1021A0001F910F91FF90EF90DF90CF90BF90AF9075
:1021B0009F908F9008950091460210914702E5E0AC
:1021C0006E9FE0011124C45DDC4F4801F12CF5E065
:1021D000E12CFF1629F0CE010196FE01E490EC01FE
:1021E000B12CA12C4E2D4170B6016A0D7B1DC4018E
:1021F0000E94420FE694FFEFAF1ABF0A88E0A816CC
:10220000B10481F7F394EFEF8E1A9E0AF6E0FF1205
:10221000DECF0A5F1F4F1093470200934602BCCFE8
:10222000DF92EF92FF920F931F93CF93DF937C0186
:10223000D22E8B01040F111DEB0177FF02C0D0E0FD
:10224000C0E0C8010134110514F080E490E0C81723
:10225000D9073CF44D2DBE01C7010E94420F2196C3
:10226000F0CFDF91CF911F910F91FF90EF90DF9012
:1022700008952F923F924F925F926F927F928F922A
:102280009F92AF92BF92CF92DF92EF92FF920F9305
:102290001F93CF93DF9300D000D000D0CDB7DEB72F
:1022A0006C01762E542E4901602E98E0A92EB12C97
:1022B000611103C089E0A82EB12CCE0101967C01EA
:1022C0008E010D5F1F4F9E012B5F3F4FA401652DB7
:1022D000872D0E94170A09811A81552011F1B40136
:1022E000990C880B990B0E94C03120E030E040E04F
:1022F0005FE30E941F321B012C0120E030E0A901A6
:102300000E94FA3420E030E040E05FE387FD0CC03B
:10231000C201B1010E948E330E946C34C616D706EA
:1023200044F48D809E8009C0C201B1010E948D33AA
:10233000F3CF8B809C80C61AD70ACA9CB001CB9C75
:10234000700DDA9C700D1124060F171FC40104973D
:102350006620B1F061E070E0711002C062E070E0F0
:10236000060F171F6C01C6012FEFC21AD20AC8143C
:10237000D90491F020E045E0B8010E941011F3CF9C
:1023800061E070E0711002C062E070E0600F711FE8
:1023900046EB5FE00E94100A26960FB6F894DEBF67
:1023A0000FBECDBFDF91CF911F910F91FF90EF90A6
:1023B000DF90CF90BF90AF909F908F907F906F9065
:1023C0005F904F903F902F9008950F93CF93DF939E
:1023D000EC019E816A3059F48D818C836985960F5A
:1023E0009E8381E090E0DF91CF910F910895262F99
:1023F00061E0690F2A3398F4203378F5273249F1E8
:1024000040F4213261F198859C5F8C81890F8C8327
:10241000E8CF2C3231F12E32B1F72FE309C021344D
:1024200090F32B35C0F08FE9820F27548A3158F78B
:10243000062E000C770B8C81082E000C990B3F8127
:102440000AEF313009F00BEF42E252E00E945008EF
:10245000DACF21E4EDCF2154EBCF2C5FE9CF2EE38F
:10246000E7CF20E4E5CF0F93CF93DF93EC019E817C
:102470006A3059F48D818C836985960F9E8381E043
:1024800090E0DF91CF910F910895262F61E0690FC1
:102490002A3398F4203378F5273249F140F4213279
:1024A00061F198859D5F8C81890F8C83E8CF2C32F8
:1024B00031F12E32B1F72FE309C0213490F32B35DF
:1024C000C0F08FE9820F27548A3158F7062E000C8E
:1024D000770B8C81082E000C990B3F810AEF31306D
:1024E00009F00BEF4AE551E00E945008DACF21E4F1
:1024F000EDCF2154EBCF2C5FE9CF2EE3E7CF20E4E3
:10250000E5CFECE8F2E084EA92E030E020E04191AF
:10251000519161917191240F351F8E179F07B9F763
:1025200080915B0290915C02821B930B0895E09175
:10253000B002F091B1023197E731F10508F036C0F1
:10254000EC55FD4E0C940F35BB12D612C112D612AB
:10255000BE12C412C712D612D612BB12CA12D6129B
:10256000D612D612D612D612D612D112D112D61235
:10257000BE12D612BE1282E090E0089581E090E093
:10258000089583E090E0089584E090E0089585E068
:1025900090E008958091A6029091A7020497029777
:1025A00028F480916B0290916C02089590E080E095
:1025B0000895CF93C82F84E00E94370F811107C080
:1025C000CC23B1F088E00E94370F882389F0109265
:1025D000B6020E9497129093B5028093B402809144
:1025E000A6029091A7029093B1028093B00281E07D
:1025F000CF910895E8E6F7E08AE48583848387E352
:10260000868369ED70E0CF010E94D90E8BE490E0E3
:102610000E94041087E690E00C940410CF92DF92A1
:10262000EF92FF920F931F93CF93DF9346E770E0F3
:1026300060E085E090E00E94190846E76FE370E0F3
:1026400085E090E00E94190821E046E365E070E033
:1026500090E080E00E94101121E046E365E070E028
:102660008FE790E00E94101141E065E070E085E0A6
:1026700090E00E94600F42E065E070E08AE790E041
:102680000E94600F44E06AE370E08AE790E00E94F5
:10269000600F48E06AE370E085E090E00E94600F20
:1026A00080916D02C6E2D7E0811122C00AE010E0FD
:1026B000F12CE12C8AE0C82ED12C80916E029091F1
:1026C0006F02E816F90684F58FEFE81AF80AD0923F
:1026D0004702C09246021093490200934802BE018D
:1026E0008CE797E00E94190E065F1F4F2696E5CFF4
:1026F0001AE0F12CE12C0AE080916E0290916F02B9
:10270000E816F9068CF40093770700937607109388
:102710007807BE0182E797E00E94190E8FEFE81A52
:10272000F80A175F2696E8CFDF91CF911F910F919E
:10273000FF90EF90DF90CF900895BC01E2E7F7E0C3
:1027400096E0958394838CE08683CF010C94190ED8
:1027500090E080E008958F929F92AF92BF92EF92A7
:10276000FF920F931F93CF93DF93CDB7DEB7A1975F
:102770000FB6F894DEBF0FBECDBF7C01FA01CB01CE
:1027800019A2223008F42AE08E010F5D1F4F822E1D
:10279000912CB12CA12CBF01A50194010E945C33A6
:1027A000F901CA016A3074F5605DD8016E938D013C
:1027B000232B242B252B79F790E080E0109789F0CC
:1027C000FD0101900020E9F73197AF014A1B5B0B37
:1027D000D701ED91FC910280F381E02DB801C70192
:1027E0000995A1960FB6F894DEBF0FBECDBFDF915D
:1027F000CF911F910F91FF90EF90BF90AF909F905E
:102800008F900895695CD1CFCF92DF92EF92FF92C3
:102810000F931F93CF93DF9377FF21C06A017B0152
:10282000EC01E881F9810190F081E02D6DE20995DC
:102830008C0144275527BA014C195D096E097F099F
:102840002AE0CE010E94AB13800F911FDF91CF9140
:102850001F910F91FF90EF90DF90CF9008952AE0A5
:10286000DF91CF911F910F91FF90EF90DF90CF906C
:102870000C94AB13CF93DF93CFE1D0E020E04AE09C
:1028800067E170E0CE010E9410112196CF36D1058C
:10289000A9F783E2809377078093760788E1809396
:1028A00078074091570250915802609159027091F7
:1028B0005A0282E797E0DF91CF910C940414BC0197
:1028C000E2E7F7E09AE09583948388E18683CF017D
:1028D0000E94190E48E566E170E08EE190E00E94EA
:1028E000190848E561E270E08EE190E00E94190865
:1028F00021E04CE066E170E08EE190E00E94101172
:1029000021E04CE066E170E085E790E00E94101164
:102910000E943A1442ED50E068E170E08FE690E0EA
:102920000C94100ACF92DF92EF92FF920F931F93B5
:10293000CF93C82F8B0169017A016E5F7F4F4BECFB
:1029400050E00E94100ACA5FE2E7F7E0C583C48343
:102950000683B701A601CF01CF911F910F91FF9080
:10296000EF90DF90CF900C940414CF93DF9380917D
:10297000B0029091B1024297029768F5C8E2D0E0A8
:1029800020E047E065E270E0CE010E941011219640
:10299000CF37D105A9F7E0916B02F0916C02EE0FF1
:1029A000FF1FEE0FFF1FEC58FD4F20813181428148
:1029B0005381609157027091580280915902909111
:1029C0005A020E94FF349B01AC0165E270E088E28C
:1029D00090E00E949214DF91CF910C943A14CF931F
:1029E000DF93EC0188819981009711F00E94B13545
:1029F000198218821D821C821B821A82DF91CF915C
:102A00000895FC0180819181009711F00C94B135FB
:102A10000895CF93C82F8091AE029091AF02019696
:102A20009093AF028093AE02109256020E94F03053
:102A300021EE3EE240E050E00E94F3326058714CDB
:102A40008F4F9F4F6093740270937502809376024C
:102A5000909377020E94F03029E53BE140E050E09E
:102A60000E94F33268577C4E8F4F9F4F60937802DD
:102A70007093790280937A0290937B020E94F030E7
:102A800023E230E040E050E00E94F3329B01AC01D1
:102A9000265F3F4F4F4F5F4FA4E6B0E00E941233D6
:102AA00060937C0270937D0280937E0290937F02FC
:102AB0000E94F0302BE230E040E050E00E94F33220
:102AC0009B01AC012F5D3F4F4F4F5F4FAAE0B0E03D
:102AD0000E9412336093800270938102809382027D
:102AE000909383020E94F03020E130E040E050E01B
:102AF0000E94F3329B01AC01295F3F4F4F4F5F4F64
:102B0000AAE0B0E00E9412336093840270938502C1
:102B100080938602909387020E94F03025E030E097
:102B200040E050E00E94F3329B01AC012F5F3F4F29
:102B30004F4F5F4FAAE0B0E00E94123360938802CB
:102B40007093890280938A0290938B02CC23C1F107
:102B500060916302709164028091650290916602B7
:102B60000E94C0312DEC3CEC4CE85FE30E941F3228
:102B70000E94A2340E946C346093630270936402DA
:102B8000809365029093660260915F02709160028B
:102B900080916102909162020E94C03124E13EEA7C
:102BA00047E85FE30E941F320E94A2340E946C3407
:102BB00060935F027093600280936102909362025F
:102BC0001092B602CF91089522E030E03093B10226
:102BD0002093B00240ED57E060E070E04093670260
:102BE000509368026093690270936A0248E853E167
:102BF00060E070E04093630250936402609365026A
:102C00007093660210925F0210926002109261024D
:102C1000109262021092A5021092A40210925E021B
:102C200010925D0224E630E030935C0220935B0258
:102C300022E330E03093710220937002ECE8F2E07E
:102C4000119211921192119222E0E43AF207C1F727
:102C500001969093AD028093AC021092AF02109255
:102C6000AE0280E00C9409159F92AF92BF92CF9272
:102C7000DF92EF92FF920F931F93CF93DF935C014C
:102C80007B018B01D0E0C0E0F80191908F016501DC
:102C9000CC0EDD1EC6010E94DD32981621F0692D92
:102CA000C6010E94E5322196C430D10569F7C701FB
:102CB000DF91CF911F910F91FF90EF90DF90CF9018
:102CC000BF90AF909F9008950C94DD32CF92DF9229
:102CD000EF92FF920F931F93CF93DF93EB017B0152
:102CE00024E0E20EF11C8B016C01C61AD70AC60162
:102CF000800F911F0E94DD32F80181938F01EE1544
:102D0000FF05A9F7CE01DF91CF911F910F91FF90A1
:102D1000EF90DF90CF9008950F931F93CF93DF93A1
:102D20008C01EB01FC01808191810097E1F06881C9
:102D3000798161157105A9F0428153812C813D8112
:102D40004217530770F00E9409378C819D81F8016A
:102D5000958384831D821C82DF91CF911F910F91F7
:102D600008950E94B13588819981F801918380830B
:102D70008A819B81938382838C819D8195838483C7
:102D8000198218821B821A82E5CF0F931F93CF936B
:102D9000DF93EC0188819981009759F02A813B816A
:102DA0002617370730F081E0DF91CF911F910F9107
:102DB00008958B016F5F7F4F0E943A36009759F05C
:102DC000998388831B830A832C813D81232B59F7A8
:102DD000FC011082E8CF80E0E7CFEF92FF920F93E3
:102DE0001F93CF93DF93EC017B01CB010E944F3106
:102DF0000097A9F00C811D81080F191FB801CE01A1
:102E00000E94C516882361F0288139818C819D81BB
:102E1000B701820F931F0E9448311D830C8381E00C
:102E2000DF91CF911F910F91FF90EF900895EF9256
:102E3000FF920F931F93CF93DF93FB01E080F1800C
:102E4000E114F10441F480E0DF91CF911F910F91E3
:102E5000FF90EF9008950481158101151105B1F0DF
:102E6000EC018C819D81080F191FB801CE010E94D1
:102E7000C516882341F3288139818C819D81B70152
:102E8000820F931F0E9409371D830C8381E0DCCFE2
:102E9000EF92FF920F931F93CF93DF93EC018B017F
:102EA0006115710551F0CB010E944F317C01BC01CD
:102EB000CE010E94C51681110BC0CE010E94EF14F5
:102EC000CE01DF91CF911F910F91FF90EF90089568
:102ED000FD82EC82B801888199810E944831F0CF4F
:102EE000FC011182108213821282158214820C94CA
:102EF0004817CF93DF93EC016230710501F148F47C
:102F00006115710581F061307105B1F06FE271E01A
:102F10000CC064307105C9F0A8F065307105B1F7D7
:102F200060E371E002C06EE471E0CE010E947017B0
:102F3000CE01DF91CF91089566E471E0F6CF61E4B0
:102F400071E0F3CF6CE371E0F0CF66E371E0EDCFB9
:102F5000CF93DF93EC016230710501F148F4611504
:102F6000710581F061307105B1F065EE70E00CC063
:102F700064307105C9F0A8F065307105B1F766EEEF
:102F800070E002C062E271E0CE010E947017CE01D3
:102F9000DF91CF91089565E171E0F6CF6BE071E0CC
:102FA000F3CF6EEF70E0F0CF63EF70E0EDCFEF9214
:102FB000FF920F931F93CF93DF93EC017B018A0164
:102FC000BA010E94C51681110BC0CE010E94EF14F8
:102FD000CE01DF91CF911F910F91FF90EF90089557
:102FE0001D830C83B701888199810E940937F0CF36
:102FF000FB0101900020E9F73197AF01461B570B09
:103000000C94D7170F931F93CF93DF93CDB7DEB7F1
:1030100062970FB6F894DEBF0FBECDBF8C01CB0117
:10302000F8011182108213821282158214824AE002
:10303000BE016F5F7F4F0E945831BE016F5F7F4FAF
:10304000C8010E94F81762960FB6F894DEBF0FBE53
:10305000CDBFDF91CF911F910F9108950F931F93D3
:10306000CF93DF93CDB7DEB7A2970FB6F894DEBF4C
:103070000FBECDBF8C01CB01BA01F80111821082C5
:1030800013821282158214822AE0AE014F5F5F4FD5
:103090000E946331BE016F5F7F4FC8010E94F81725
:1030A000A2960FB6F894DEBF0FBECDBFDF91CF91D1
:1030B0001F910F9108952F923F924F925F926F92BE
:1030C0007F928F929F92AF92BF92CF92DF92EF92B8
:1030D000FF920F931F93CF93DF93CDB7DEB7629725
:1030E0000FB6F894DEBF0FBECDBF2C019E012F5F3F
:1030F0003F4F490139011C01D12CC12C10E000E0E7
:10310000B12CA12CF10141915191619171911F015B
:10311000CE010D960E942E18E988FA88CE010D96F0
:103120000E940115B601CE010D960E94791789897A
:103130009A89E80EF91EFFEFEF1AFF0AF301E192F8
:10314000F1923F01CE010D960E940115F3E0CF16DA
:10315000D1040CF03FC0AE14BF040CF457012FEFA4
:10316000C21AD20A36E0C316D10461F684E4C82E2E
:1031700087E0D82EF12CE12C150183E0E816F1044C
:103180000CF01801B701CE010D960E947917BE010F
:10319000635F7F4FC6010E948C16CE010D960E9480
:1031A000011568E571E0C6010E94ED16712C612CD5
:1031B000F401808191819101281B390B62167306FD
:1031C00074F466E571E0C6010E94ED163FEF631AE4
:1031D000730AEECF0E151F0514F68701C0CFF2015A
:1031E00041915191619171912F01CE010D960E94F3
:1031F0002E18BE01635F7F4FC6010E941717CE01D4
:103200000D960E940115FFEFEF1AFF0A26E0C20E8D
:10321000D11C32E0830E911C86E0E816F10409F01F
:10322000ABCFF092AB02E092AA0281E08093A802B9
:103230000A0D1B1D073111050CF480E08093A902D3
:1032400062960FB6F894DEBF0FBECDBFDF91CF916F
:103250001F910F91FF90EF90DF90CF90BF90AF90B4
:103260009F908F907F906F905F904F903F902F90A6
:103270000895EF92FF920F931F93CF93DF9300D0A7
:1032800000D000D0CDB7DEB78C019CE3E92EF12C45
:1032900020E04CE069E070E0C7010E9410118FEF60
:1032A000E81AF80A80E8E816F10491F7000F111FF8
:1032B000000F111FF801E457FD4F408151816281D9
:1032C0007381CE0101960E942E188D818195880F01
:1032D000880F845A80936D0780936C078DE08093EC
:1032E0006E0748E050E06CE571E088E697E00E94E8
:1032F000FD0EBE016F5F7F4F88E697E00E94190EBA
:10330000CE0101960E94011526960FB6F894DEBFF5
:103310000FBECDBFDF91CF911F910F91FF90EF9026
:103320000895EF92FF920F931F93CF93DF9300D0F6
:1033300000D000D0CDB7DEB78091B0029091B1023D
:103340000A9709F05EC00E9481128C01BC01CE0177
:1033500001960E940218ED80FE80CE0101960E9427
:10336000011581E080936D0780936C0710926E07C2
:1033700064EC70E088E697E00E94D90E40915D020F
:1033800050915E02052E000C660B770B88E697E0E5
:103390000E94041487E190E08E199F09880F991FFD
:1033A000880F991F80936D0780936C0710926E07AA
:1033B0006AEB70E088E697E00E94D90EA801110F31
:1033C000660B770B88E697E00E94041410E000E09B
:1033D00021E041E068E070E0C8010E9410110F5F39
:1033E0001F4F00381105A1F726960FB6F894DEBFDF
:1033F0000FBECDBFDF91CF911F910F91FF90EF9046
:10340000089540916702509168026091690270913D
:103410006A02CE0101960E942E18ED80FE80CE0138
:1034200001960E94011500E210E00E191F09000F1D
:10343000111F000F111F8091B0029091B1029C01E9
:10344000265031092230310508F052C021E0209386
:103450006D0720936C0710926E0760EB70E0069783
:1034600011F465EB70E088E697E00E94D90E4BEC12
:1034700050E061E070E083E190E00E94100A89E191
:1034800080936D0780936C0710926E078091B00255
:103490009091B102069719F5409163025091640230
:1034A000609165027091660288E697E00E940414BC
:1034B0004BEC50E061E070E0C80106970E94100AF2
:1034C00000936D0700936C0710926E07409167029E
:1034D000509168026091690270916A0273CF4091C5
:1034E0005F02509160026091610270916202DCCFD4
:1034F00081E080936D0780936C0710926E076CEAF1
:1035000070E088E697E00E94D90E8EE080936D0708
:1035100080936C0710926E074091AE025091AF02FB
:10352000052E000C660B770BBFCF1F920F920FB6C4
:103530000F9211248F939F938091E1009091E1006D
:10354000937F9093E10083FF0FC01092E90091E018
:103550009093EB001092EC0092E39093ED001092A8
:10356000D50298E09093F00082FF22C093E0909300
:10357000E9009091F200992319F09AE39093E80002
:103580009091C602992341F09091C6029150909378
:10359000C602911101C05D9A9091D402992341F025
:1035A0009091D40291509093D402911101C0289A25
:1035B00084FF18C08091E2008E7E81608093E200DB
:1035C0008091E1008F7E8093E1008091C7028E7E22
:1035D00080618093C7029F918F910F900FBE0F90D3
:1035E0001F90189580FFF7CF8091E2008E7E80615A
:1035F0008093E2008091E1008E7E8093E1008091D3
:10360000C7028E7E8160E5CF1F920F920FB60F9298
:103610001124CF92DF92EF92FF920F931F932F937B
:103620003F934F935F936F937F938F939F93AF934A
:10363000BF93EF93FF93CF93DF93CDB7DEB76C9734
:10364000DEBFCDBF1092E9008091E80083FF25C066
:1036500068E0CE0145960E942E0D82EF8093E8002F
:103660008D8987FF39C09091E80090FFFCCF982F9B
:10367000907609F034C19E894F89588D2F89F88C36
:10368000911131C0803861F58091C5028093F100BD
:103690001092F1008EEF8093E8006C960FB6F894CC
:1036A000DEBF0FBECDBFDF91CF91FF91EF91BF91F4
:1036B000AF919F918F917F916F915F914F913F91CA
:1036C0002F911F910F91FF90EF90DF90CF900F906F
:1036D0000FBE0F901F9018959EEF9093E800C7CFF4
:1036E0001092F100D5CF913059F48111D3CF4130F0
:1036F000510581F68091C5028D7F8093C502CACFA6
:10370000933049F48111C6CF4130510519F68091AB
:10371000C5028260F2CF953041F48091E80080FFCD
:10372000FCCF20682093E300B5CF963009F0A9C004
:103730000B8D1C8D22E01092E9001092C3021092B2
:10374000C202F2122EC01092C1021092C0020E9458
:10375000FD0C1F8299E09983FA8291E09E8390EAA2
:1037600098879AEF99872091C2023091C302275F10
:103770003F4F3C832B838D831092E9001092C3024C
:103780001092C2021093C1020093C00249E050E0BF
:10379000BE016F5F7F4F80E00E94D70C0E94FD0C3E
:1037A00079CF1093C1020093C0020E94140CDC0177
:1037B00012960D911C910115110509F451C1D80102
:1037C000ED91FC910480F581E02DBE016B5E7F4F91
:1037D000C8010995009709F03EC1F80100851185DF
:1037E000EACFF3E0FF120EC08F89882309F440C0AE
:1037F000823061F440E860E185EA9FE00E94801D2C
:10380000811148CF81E28093EB0047CF813029F4CA
:1038100040E86BE089E99FE0F1CF833099F70E949F
:10382000140CDC011296ED90FC908E010F5F1F4F7F
:103830006801E114F10479F0D701ED91FC91068063
:10384000F781E02DB801C7010995080F111DF70197
:10385000E084F184EECFD8011C92F60101900020A3
:10386000E9F73197BF016C197D0940E0C601C6CF69
:1038700063E87FE0FB01449150E080E80E94D70CB0
:1038800009CF973009F4BECF983021F481E08093BE
:10389000F10000CF993009F0FDCE837009F0B2CF6E
:1038A000E0E2F1E081E031E096E32191222371F042
:1038B0008093E9003093EB00DF0111972C91209366
:1038C000EC009093ED008F5F873079F78EE780935F
:1038D000EA001092EA008F898093D502DBCE8B8DAF
:1038E0009C8D1092E9001092C3021092C202909334
:1038F000C1028093C002898D811192C08E899D89F9
:10390000913A49F4813209F07DCF47E050E06DE013
:1039100071E080E0B3CF913209F074CF833269F463
:103920008F89988DB0E0A0E08093090190930A01FF
:10393000A0930B01B0930C01ADCE803269F480915D
:10394000E80082FFFCCF67E08DE091E00E942E0D41
:103950008BEF8093E8009ECE823209F09BCE8F8958
:1039600080931401EEEFFFE7859194918B3F9C4D7E
:1039700051F1E0E0F8E080910D0190910E01A091ED
:103980000F01B0911001803B9440A105B105F1F405
:103990008091140180FD1AC0EE3F8AE0F80789F596
:1039A00087E797E791838083809160008093C402CA
:1039B00088E19BE00FB6F894A895809360000FBE55
:1039C0009093600067CEEEEFFAE0D5CF80819181D1
:1039D0008737974709F05ECEA8958091600088618F
:1039E000809360008091C40280936000EE3F2AE0E3
:1039F000F20789F08091FE0A9091FF0A91838083FB
:103A000049CE808191818737980751F29093FF0AC0
:103A10008093FE0AC5CF1092FF0A1092FE0A3ACE9A
:103A20000E94140CDC0112960D911C9101151105D8
:103A300009F4E8CED801ED91FC910190F081E02DE0
:103A4000BE016B5E7F4FC8010995811123CEF8013D
:103A500000851185EBCF181619060CF41BCED2CEBB
:103A6000F1E0FF12BECE67E87FE004CF1F920F9215
:103A70000FB60F9211242F933F938F939F93AF9381
:103A8000BF938091B8029091B902A091BA02B0910F
:103A9000BB023091B70223E0230F2D3758F5019672
:103AA000A11DB11D2093B7028093B8029093B90273
:103AB000A093BA02B093BB028091BC029091BD0268
:103AC000A091BE02B091BF020196A11DB11D8093CD
:103AD000BC029093BD02A093BE02B093BF02BF91FF
:103AE000AF919F918F913F912F910F900FBE0F90AB
:103AF0001F90189526E8230F0296A11DB11DD2CF65
:103B0000EF92FF920F931F93CF93DF93F82E192F0D
:103B1000E62E042F81E0860F880F0E94A90C83E017
:103B20000E94A90CCF2DD12FEC0EFD2EF11CCE152D
:103B3000DF05B9F007FF13C0FE0184910E94A90CB4
:103B4000182F80E00E94A90C812321968111EFCFCC
:103B5000DF91CF911F910F91FF90EF900895888191
:103B6000EDCF81E0F5CFCF93DF931092D90610927D
:103B7000D80688EE93E0A0E0B0E08093DA06909358
:103B8000DB06A093DC06B093DD068AE291E0909319
:103B9000D7068093D6068FEF9FEF9093E30680932E
:103BA000E20610927F0710927E0784E591E09093E1
:103BB0007D0780937C07109275071092740788E444
:103BC00091E0909373078093720798E090937B073E
:103BD00081E080937A07109277071092780710920D
:103BE00076078093790710926B0710926A072CE38F
:103BF00031E03093690720936807909371078093B1
:103C0000700710926D0710926E0710926C078093E8
:103C10006F07C4E4D7E0198218821B821A821D82C2
:103C20001C8250E040E064E671E0CE010E94D717AC
:103C3000269687E0C836D80771F7C6E2D7E0198222
:103C400018821B821A821D821C8250E040E064E6CA
:103C500071E0CE010E94D717269687E0C434D807BA
:103C600071F7DF91CF910895CF93DF93CDB7DEB792
:103C70002D970FB6F894DEBF0FBECDBF789484B5F4
:103C8000826084BD84B5816084BD85B5826085BD58
:103C900085B5816085BD80916E00816080936E00E6
:103CA00010928100809181008260809381008091D8
:103CB0008100816080938100809180008160809389
:103CC00080008091910082608093910080919100AA
:103CD000816080939100809190008160809390003A
:103CE0008091C10084608093C1008091C100826096
:103CF0008093C1008091C10081608093C100809158
:103D0000C30081608093C3008091C0008260809373
:103D1000C0008091C20081608093C20080917A00CF
:103D2000846080937A0080917A00826080937A0028
:103D300080917A00816080937A0080917A00806817
:103D400080937A001092D5021092C5021092C70299
:103D50008091D70081608093D70080EA8093D8005B
:103D600089B5806189BD89B5826089BD09B400FECD
:103D7000FDCF61E070E080E090E00E94600D8091F6
:103D8000D8008F7C80618093D8008091E000807F94
:103D90008093E0008091E1008E7E8093E1008DE0D1
:103DA0008093E200559A209A81EC80937C0085B143
:103DB000806F85B984B1877E84B984B1876E84B9F8
:103DC0005E9A5F988AB1806D8AB9769A6E9881B34F
:103DD000806F81BB899880B38D7080BB80E58CBD7E
:103DE00081E08DBD85E090E00E942A0F5F9A85E01A
:103DF00090E00E942A0F5E985C98ECE2F8E089E37C
:103E000098E024912EBD00000DB407FEFDCF319641
:103E10008E179F07B1F75C9A81E8809364008091C8
:103E2000650081608093650081E090E00E946416E7
:103E300081FF0EC0082F0470F02E82FD2E9801EF36
:103E40001FEF0E942F0F86FF83C02E9A2F9A2D9A64
:103E500082E480930001809164008E7F80936400EF
:103E600080917A00806480937A0080917A0086FD48
:103E7000FCCF00917800109179000E943B0DAB01BE
:103E8000BC01C801B0E0A0E0DC01992788276C01E3
:103E90007D01C40ED51EE61EF71EC701B601209196
:103EA000640021602093640061157105810591050E
:103EB00011F00E943F311092B1021092B0021092A4
:103EC000B6028E010F5F1F4F780101E110E07E2CDA
:103ED0006F2CC8010E94DD32D7018D937D010F5FE9
:103EE0001F4F06311105A9F765E671E0872D962D64
:103EF0000E94003715E6E12E11E0F12E01E110E0FD
:103F0000892B09F07EC065E071E086E190E00E94B7
:103F1000661661E071E08AE190E00E9466168FB754
:103F2000F8944091B8025091B9026091BA02709130
:103F3000BB028FBF80914402882309F480C0109295
:103F4000440280E090E0892B51F30E940000E7CF0B
:103F5000FF2029F00430110511F42E9A2F9881E0EA
:103F60000E940A0849E358E0B80184E190E00E9409
:103F7000100A80E00E940A088FE090E00E942A0F59
:103F80000F5F1F4F0931110509F05BCFFF2011F0C2
:103F90002F9A2D9880E991E00E942A0F2D9A81E0B6
:103FA00090E00E94641680FF53CF8AE090E00E9468
:103FB00064169FEF980F9E3F08F04ACF22E330E04F
:103FC000309347022093460228E330E030934902C1
:103FD000209348020BE010E0682F8CE797E00E94E6
:103FE000AD10C8010E9464160F5F1F4F013111050B
:103FF00099F780E00E940A0888EE93E00E942A0F59
:1040000027CFF701D1907F01C8010E94DD32D81679
:1040100021F06D2DC8010E94E5320F5F1F4F063160
:10402000110579F765E071E086E190E00E943416B1
:1040300061E071E08AE190E00E94341670CF8091D7
:104040004502F42FF81B8F2F90910001F91748F4C7
:104050008F5F891708F075CF81E083BF889513BE05
:1040600070CF81E0809344024093450280914202E8
:104070009091430201969093430280934202809173
:104080004B0280934A020E942F0F80934B02809133
:10409000B6028111E4C02091B0023091B102E6ED88
:1040A000F2E081118FEF00248193819381938193BA
:1040B0000394D1F7109249021092480210924702DD
:1040C000109246028091B4029091B5029093B3028F
:1040D0008093B2021092B5021092B40222303105E0
:1040E00089F42091AE023091AF028091AC029091A0
:1040F000AD022817390734F088E190E09093B102BF
:104100008093B0028091B0029091B1028931910503
:1041100008F083C5FC01E157FF4D0C940F35A82032
:104120000A2156210022C621C6217A22A422BD22BC
:104130002023A721AD23AD23AD23AD23B923E52350
:10414000822304240424A624A624A624A62413251A
:1041500047EC5EE070E060E090E080E00E94100AD2
:1041600047EC5EE070E060E082E690E00E94100ABA
:104170008AE290E090934702809346028AE090E0C2
:1041800090934902809348026EEB7EE08CE797E0C3
:104190000E94D90E87E680936D0780936C078AE3AF
:1041A00080936E0767EB7EE088E697E00E94D90E69
:1041B00068EA7EE084E497E00E9448176AE97EE0BE
:1041C0008AE497E00E9448176EE87EE080E597E079
:1041D0000E94481783E090E09093AB028093AA027C
:1041E00081E08093A9021092A80243E050E060E0D1
:1041F0000E94270E2091AA023091AB0200E040916C
:10420000A8026091A9028091B2029091B3020E942B
:10421000391122C00E940E13209105013091060130
:10422000409107015091080163E170E08AE090E05D
:104230000E949214209101013091020140910301EA
:104240005091040167E270E08AE090E00E949214CD
:104250001092A7021092A60281E08093B602C0904D
:10426000B002D090B102B9E1CB16D10408F077C505
:10427000F601E35CFE4D0C940F352A265C2C2A26B1
:104280002A262A262A262A262A26E82C5C2C5C2C7A
:104290005C2C602C602C602C5C2C5C2C602CE12D48
:1042A000E12DE12DE12DE12DE12D5C2C0E949119F4
:1042B0006091A4027091A502872D962D0E94A817E7
:1042C000872D962D0E949D13872D962D0E940115F6
:1042D00064E87EE084E497E00E94481769E77EE0A6
:1042E0008AE497E00E9448176EE67EE080E597E05A
:1042F0000E9448176AE67EE086E597E00E9448172C
:104300008091A4029091A502892BF1F46FE57EE0E3
:104310008CE597E00E9448176AE57EE082E697E028
:104320000E94481786E090E09093AB028093AA0227
:104330001092A90281E08093A8024091AA025091B4
:10434000AB0261E080E054CF84E090E0EDCF0E94CA
:1043500091196FE47EE0872D962D0E947017872DAE
:10436000962D0E949D13872D962D0E9401158CE895
:1043700092E00E945B184091AA025091AB026091BA
:10438000A8028091A9020E94270E66CF0E9491196F
:104390008091B0029091B10265E47EE0049711F043
:1043A0006AE37EE0872D962D0E947017872D962D4B
:1043B0000E949D13872D962D0E94011584E792E09F
:1043C0000E945B184091AA025091AB026091A80232
:1043D0008091A9020E94270EE090B202F090B302F1
:1043E0002091AA023091AB0200E04091A8026091B6
:1043F000A902C7010E943911C7010E9439192CCFA7
:104400000E94911960E37EE0CE0107960E9470172A
:104410006091A4027091A502872D962D0E94A81785
:10442000672D762DCE0107960E941717872D962DA2
:104430000E9401151A8219821C821B821E821D8213
:104440006F8178856115710531F04B855C85872D0D
:10445000962D0E94D717872D962D0E949D13872D8C
:10446000962D0E940115B4E4EB2EB7E0FB2E70E010
:1044700060E08B010F5F1F4F8091A4029091A50215
:10448000681779070CF0B801872D962D0E94A817A0
:10449000672D762DC7010E948C16872D962D0E94C0
:1044A000011526E0E20EF11CB8010530110509F7EF
:1044B0001093AB020093AA0281E08093A90280933B
:1044C000A80245E050E061E00E94270E2091AA0278
:1044D0003091AB0200E04091A8026091A902809166
:1044E000B2029091B3020E943911CE0107960E9448
:1044F0000115B2CE0E94911965E27EE0872D962DBE
:104500000E947017872D962D0E949D13872D962D42
:104510000E9401156AE17EE084E497E00E9448175A
:104520006DE07EE08AE497E00E94481782E090E028
:104530009093AB028093AA021092A9021092A80253
:1045400042E050E060E0FECE0E94911968E07EE01B
:10455000872D962D0E947017872D962D0E949D13F2
:10456000872D962D0E9401156AEF7DE084E497E087
:104570000E9448176BEE7DE0D5CF6CED7DE086E2C2
:1045800097E00E94481761ED7DE08CE297E00E9481
:1045900048176091720270917302872D962D0E94C8
:1045A0000218672D762D8CE297E00E941717872D51
:1045B000962D0E9401156BEC7DE08CE297E00E9445
:1045C000ED166AEB7DE082E397E00E9448176CEA03
:1045D0007DE088E397E00E94481760917002709137
:1045E0007102872D962D0E940218672D762D88E383
:1045F00097E00E941717872D962D0E94011584E0E1
:1046000090E090936F0280936E0210926D020E9470
:104610000E1382E480936D0780936C0787E3809389
:104620006E076EEB7CE088E697E00E94D90E83E48B
:1046300090E00E94041087E690E00E9404100CCEE7
:104640000E94F0306B017C016EEA7CE086E297E02C
:104650000E94481767EA7CE08CE297E00E944817C6
:1046600088E090E09093A7028093A60283E090E018
:1046700090936F0280936E0210926D02C701B60193
:1046800022E030E040E050E00E94F332672B79F402
:1046900062EA7CE08CE297E00E94ED1669E97CE03A
:1046A00082E397E00E9448170E940E13D5CD62E97D
:1046B0007CE08CE297E00E94ED1668E87CE082E303
:1046C00097E00E94481780917002909171020397C1
:1046D0009093710280937002181619062CF368E704
:1046E0007CE088E397E00E94481784E090E0909394
:1046F0006F0280936E0288E190E09093A70280930E
:10470000A602D2CF6AE97DE086E297E00E944817D0
:104710006CE87DE08CE297E00E9448176DE77DE051
:1047200082E397E00E94481761E77DE088E397E025
:104730000E94481784E090E090936F0280936E028D
:1047400010926D020E940E130E94FA1282E090E015
:104750009093A7028093A6027FCD0E940E138091B2
:10476000B0029091B1020B9709F476CD0E94FA1233
:1047700073CD6AE671E086E297E00E94F8176DE774
:1047800071E08CE297E00E94F81762E971E082E341
:1047900097E00E94F81766EA71E088E397E00E94CC
:1047A000F81768EB71E08EE397E00E94F81785E058
:1047B00090E090936F0280936E0281E080936D028F
:1047C0000E940E1380E190E0C3CF64E671E086E2C0
:1047D00097E00E94F8176CEC71E08CE297E00E9481
:1047E000F8176BED71E082E397E00E94F81783E021
:1047F00090E090936F0280936E0210926D020E947F
:104800000E1388E190E0A4CF6AE67DE0429711F0B4
:1048100064E67DE086E297E00E94481760916B02B3
:1048200070916C02872D962D0E947917672D762D39
:1048300086E297E00E941717872D962D0E9401159A
:1048400060E77DE08CE297E00E9448176FE67DE02C
:1048500082E397E00E9448178091B0029091B102E4
:1048600065E57DE0429711F06FE47DE088E397E035
:104870000E9448176BE57DE08EE397E00E944817A1
:1048800085E090E090936F0280936E0281E08093C8
:104890006D020E940E13E0916B02F0916C02EE0F1C
:1048A000FF1FEE0FFF1FEC58FD4F20813181428129
:1048B000538160912A0770912B07E5E0E69FC001C4
:1048C000E79F900D11246AE070E00F960E94921409
:1048D0008091B0029091B1024297E9F42091670271
:1048E000309168024091690250916A026EE270E074
:1048F00087E390E00E9492140E94B5146BE47DE07F
:10490000872D962D0E947017872D962D0E945F147B
:10491000872D962DECCD87E38093770780937607DC
:104920008EE280937807E0916B02F0916C02EE0FBB
:10493000FF1FEE0FFF1FE457FD4F40815181628141
:10494000738182E797E00E940414D6CF60E47DE093
:104950008431910559F063E37DE08531910531F0B3
:1049600065E27DE0469711F066E17DE086E297E042
:104970000E9448176AE47DE08CE297E00E944817A5
:1049800069E47DE082E397E00E9448178091A602E7
:104990009091A70265E07DE0069711F06DEF7CE055
:1049A00088E397E00E9448176DE07DE08EE397E092
:1049B0000E94481785E090E090936F0280936E020A
:1049C00081E080936D020E940E138091A602909167
:1049D000A7020697F9F42091630230916402409196
:1049E00065025091660265E270E082E390E00E9409
:1049F00092142091670230916802409169025091AF
:104A00006A026EE270E087E390E00E94921469EF20
:104A10007CE076CF20915F0230916002409161028C
:104A200050916202E0CF10926D0283E090E090938B
:104A30006F0280936E021092A7021092A6028090DD
:104A40005F0290906002A0906102B090620280913B
:104A5000630290916402A0916502B0916602881A87
:104A6000990AAA0ABB0A8091670290916802A091F4
:104A70006902B0916A02880E991EAA1EBB1EECE85C
:104A8000F2E004E712E064EAE62E62E0F62E2191FD
:104A9000319141915191D8016D917D918D919D916F
:104AA0008D010E94FF34860E971EA81EB91EEE16B9
:104AB000FF0669F7B7FC89C080926702909268028E
:104AC000A0926902B0926A02809167029091680296
:104AD000A0916902B0916A022091AC023091AD02BE
:104AE00011E02F31310509F079C040910501509155
:104AF00006016091070170910801481759076A077C
:104B00007B070CF010E067EE7CE086E297E00E9405
:104B1000481766EE7CE08CE297E00E94481765ED4E
:104B20007CE0111102C064ED7CE082E397E00E941A
:104B300048176AED7CE082E397E00E94ED160E9440
:104B40000E132091670230916802409169025091E2
:104B50006A0263E170E08AE090E00E949214809122
:104B6000AC029091AD024F9709F041C02091050130
:104B700030910601409107015091080167E270E011
:104B80008AE090E00E949214112309F465CB809191
:104B9000670290916802A0916902B0916A02209127
:104BA000AC023091AD022F31310551F580930501F2
:104BB00090930601A0930701B093080165E071E0AE
:104BC00086E190E00E94341647CB10926702109263
:104BD00068021092690210926A0276CF4091010138
:104BE00050910201609103017091040186CF2091E0
:104BF0000101309102014091030150910401BECFA7
:104C00008093010190930201A0930301B0930401EA
:104C100061E071E08AE190E0D5CF85E090E090938B
:104C200047028093460290934902809348026DECBC
:104C30007CE08CE797E00E94D90E4091B002509141
:104C4000B102052E000C660B770B8CE797E00E94F3
:104C5000041402CB80E80E94370F81111AC080E152
:104C60000E94370F811115C080E20E94370F811119
:104C700010C080E40E94370F81110BC088E00E94B1
:104C8000370F811106C084E00E94370F882309F492
:104C900066C0A090AA02B090AB02E090A802ED8698
:104CA000E090B202F090B30201E095014D85609171
:104CB000A902C7010E943911B5010B2C000C880B09
:104CC000990B0E94C03120E030E040E05FE30E9499
:104CD0001F321B012C0120E030E0A9010E94FA34B0
:104CE00020E030E040E05FE387FD3DC0C201B1015C
:104CF0000E948E330E946C348B0188248394912C03
:104D0000E616F7061CF042E0842E912C80E10E940A
:104D1000370F8823A9F10FEFE01AF00AEA14FB0419
:104D20003CF5F092B302E092B202E090B202F09051
:104D3000B3022091AA023091AB0200E04091A80298
:104D40006091A902C7010E9439118091B00290912F
:104D5000B1020497029718F4C7010E94391980E044
:104D60000E940A08EEC8C201B1010E948D33C2CF71
:104D700011E0A11AB108B092B302A092B202D5CF4D
:104D800080E80E94370F882371F021E0E21AF108D1
:104D9000F092B302E092B202F7FEC7CF1092B302D4
:104DA0001092B202C2CF80E40E94370F8823E1F054
:104DB000CD84CC20A9F08A94892891F4E00EF11ECC
:104DC000F092B302E092B2028091B2029091B302EB
:104DD0008A159B050CF4A9CF41E0A41AB108CBCFEA
:104DE0003FEFE31AF30AECCF80E20E94370F8823EB
:104DF000C1F0CD84CC2089F022E08216910469F4C0
:104E0000E01AF10AF092B302E092B2028091B2028B
:104E10009091B30297FF89CFC1CF31E0E31AF10837
:104E2000F1CF88E00E94370F882309F42CC5109237
:104E3000B60248E0C416D10408F077CFF601ED5D64
:104E4000F84D0C940F352B2795265F278B278A2A40
:104E5000502BB22B102C81E0E816F10461F092E0A7
:104E6000E916F10459F08EE190E0EF2809F05DCFEA
:104E70000E94E4155ACF8CE390E0FACF6BE67CE019
:104E800086E297E00E9448176AE67CE08CE297E0B1
:104E90000E9448176BE57CE082E397E00E94481788
:104EA00010926D0283E090E090936F0280936E0207
:104EB00081E090E09093B1028093B00236CF82E01F
:104EC00090E09093A7028093A602A2E0EA16F10474
:104ED000C9F04CF4E114F10491F085E090E0EA941B
:104EE000EF2841F322CFF4E0EF16F10489F06CF0E3
:104EF00087E090E015E0E116F104E1F216CF84E0DE
:104F000090E0D8CF8AE090E0D5CF83E090E0D2CF98
:104F100086E090E0CFCF8091A4029091A502E816A0
:104F2000F9061CF02FEFE21AF20AF092A502E092C5
:104F3000A40281E00E9409150E94F03024E130E0D3
:104F400040E050E00E94F3329B0142E050E0509379
:104F5000A7024093A60210926D02FB013197E13146
:104F6000F10508F0D2C2E954F84D0C940F35C8276A
:104F7000EF270E28412841286C286C289928E02822
:104F8000E028E028402940299429B529E429522A1B
:104F900065ED7BE086E297E00E94481763EC7BE0DA
:104FA0008CE297E00E9448176AEB7BE082E397E08F
:104FB0000E94481783E090E090936F0280936E0206
:104FC00082E090E0A0E0B0E08093880290938902B4
:104FD000A0938A02B0938B028BE090E06BCF69EADA
:104FE0007BE086E297E00E94481769E97BE08CE26B
:104FF00097E00E94481782E090E090936F028093C0
:105000006E028AE790E0A0E0B0E080938002909387
:105010008102A0938202B0938302DECF68E87BE036
:1050200086E297E00E9448176AE77BE08CE297E00F
:105030000E94481769E67BE082E397E00E944817E8
:105040006CE57BE088E397E00E94481784E090E0FD
:1050500090936F0280936E020E94F0302EE734E04E
:1050600040E050E00E94F3326E5A7C4F8F4F9F4FCA
:10507000609378027093790280937A0290937B0216
:10508000ABCF6CE47BE086E297E00E9448176DE3CB
:105090007BE08CE297E00E9448176FE27BE082E3BE
:1050A00097E00E94481765E27BE088E397E00E9462
:1050B000481784E090E090936F0280936E020E9404
:1050C000F03029EA31E640E050E00E94F332605BC4
:1050D000794B8F4F9F4FCCCF66E17BE086E297E024
:1050E0000E94481765E07BE08CE297E00E94481739
:1050F00062EF7AE082E397E00E94481783E090E055
:1051000090936F0280936E020E94F03021E63AEE97
:1051100040E050E00E94F3326058774C8E4F9F4F32
:105120006093740270937502809376029093770275
:1051300053CF63EE7AE086E297E00E94481767ED6E
:105140007AE08CE297E00E94481782E090E090932A
:105150006F0280936E026091670270916802809185
:10516000690290916A020E94C03120E030E040E480
:1051700050E40E94FA336B017C0120E030E0A90189
:105180000E94FA3420E030E040E05FE387FD13C086
:10519000C701B6010E948E330E946C34660F771FE0
:1051A000881F991F60936702709368028093690259
:1051B00090936A0211CFC701B6010E948D33ECCFE4
:1051C000ECE8F2E090E080E04191519161917191C1
:1051D000840F951FA2E0E43AFA07B1F7C2970CF4E6
:1051E00068C382E090E02930310539F084E090E036
:1051F0002A30310511F085E090E09093730280939E
:1052000072026BEC7AE086E297E00E94481766EC47
:105210007AE08CE297E00E944817609172027091E8
:10522000730261507109872D962D0E940218672D17
:10523000762D8CE297E00E941717872D962D0E94FD
:1052400001156EEB7AE08CE297E00E94ED1662EBBE
:105250007AE082E397E00E94481767EA7AE088E301
:1052600097E00E94481784E090E090936F0280934B
:105270006E0288E090E09093A7028093A602ACCEE5
:105280008091670290916802A0916902B0916A02D0
:10529000843F9140A105B1050CF40BC30E9481121B
:1052A00005970CF406C30E94F03023E030E040E0A4
:1052B00050E00E94F3326B0168E97AE086E297E001
:1052C0000E944817F2E0CF16D104C8F46BE77AE0E9
:1052D000CD2811F06BE67AE08CE297E00E94481747
:1052E0006BE87AE082E397E00E94481783E090E061
:1052F00090936F0280936E028CE090E0DBCD6DE5C1
:105300007AE08CE297E00E9448176FE47AE082E34B
:1053100097E00E94481766E47AE088E397E00E94ED
:10532000481784E090E0E4CF65E37AE086E297E016
:105330000E94481765E27AE08CE297E00E944817E5
:1053400063E17AE082E397E00E94481762E07AE046
:1053500088E397E00E94481784E090E090936F0202
:1053600080936E028EE090E0A5CD809167029091CF
:105370006802A0916902B0916A028C329140A10545
:10538000B1050CF496C26FEE79E086E297E00E94D8
:1053900048176FED79E08CE297E00E94481760EDC6
:1053A00079E082E397E00E94481765EC79E088E3B2
:1053B00097E00E94481784E090E090936F028093FA
:1053C0006E028DE090E076CD0E94811208970CF479
:1053D00070C20E94F03027E030E040E050E00E94D0
:1053E000F3328B010F5F1F4F0E94F03026E030E058
:1053F00040E050E00E94F3326B01FB01EE0FFF1F13
:10540000EE0FFF1FE457FD4FA801012E000C660BA5
:10541000770B80819181A281B381840F951FA61F94
:10542000B71F80839183A283B3836AEB79E086E21E
:1054300097E00E944817B801872D962D0E94021808
:10544000672D762D86E297E00E941717872D962DFF
:105450000E9401156FEA79E08CE297E00E944817FC
:10546000B601872D962D0E947917672D762D8CE237
:1054700097E00E941717872D962D0E94011569EE5F
:1054800071E082E397E00E94F8176BEF71E088E328
:1054900097E00E94F81784E090E090936F02809369
:1054A0006E029ACD69E072E086E297E00E94F817FA
:1054B00068E172E08CE297E00E94F8176AE272E01D
:1054C00082E397E00E94F81769E372E088E397E0CF
:1054D0000E94F81784E090E090936F0280936E0230
:1054E0000E94F03027E232E040E050E00E94F332C8
:1054F00066507F4F8F4F9F4F60937C0270937D0269
:1055000080937E0290937F0267CD5093B1024093C7
:10551000B0020BCC0E9481128C0194E0C92ED12CD8
:10552000D092A702C092A602F0926C02E0926B02A7
:1055300010161106DCF165E57CE086E297E00E943A
:10554000481764E57CE08CE297E00E94481764E429
:105550007CE082E397E00E9448176EE37CE088E3FA
:1055600097E00E94481760916B0270916C02872D42
:10557000962D0E947917672D762D88E397E00E947B
:105580001717872D962D0E9401156CE37CE088E3A8
:1055900097E00E94ED16D0926F02C0926E021092B8
:1055A0006D028091B0029091B10265CEF701EE0FCD
:1055B000FF1FEE0FFF1FEC58FD4F80809180A280EF
:1055C000B380609167027091680280916902909146
:1055D0006A02681579058A059B053CF566E37CE05F
:1055E00086E297E00E94481765E37CE08CE297E052
:1055F0000E94481764E27CE082E397E00E9448172B
:1056000060916B0270916C02872D962D0E94791724
:10561000672D762D88E397E00E948C16872D962DB6
:105620000E94011562E27CE0B2CF22E130E03093CB
:10563000B1022093B00210925702109258021092B9
:10564000590210925A020E94C0316B017C01C501BF
:10565000B4010E94C0319B01AC01C701B6010E9498
:10566000FA330E94A2340E946C3460934C0270930F
:105670004D0280934E0290934F02012E000C220B9C
:10568000330B06171707280739070CF04ECB00938A
:105690004C0210934D0220934E0230934F0245CBA3
:1056A00085E090E09093A7028093A602F0926C02AE
:1056B000E0926B02F701EE0FFF1FEE0FFF1FE457A2
:1056C000FD4F80819181A281B381181619061A06B7
:1056D0001B06BCF423E130E03093B1022093B0020A
:1056E00010925702109258021092590210925A02C8
:1056F00080934C0290934D02A0934E02B0934F02C0
:1057000014CB6CE17CE086E297E00E9448176BE1E5
:105710007CE08CE297E00E94481768E07CE082E33E
:1057200097E00E94481760916B0270916C02872D80
:10573000962D0E947917672D762D88E397E00E94B9
:105740008C16872D962D0E94011566E07CE088E37B
:1057500097E00E94ED1684E090E090936F028093B2
:105760006E021DCF86E090E09093A7028093A60280
:1057700010925702109258021092590210925A0237
:10578000E114F10419F1EA94EF2809F0CECA8091EE
:1057900056028823D1F16AEF7BE086E297E00E940F
:1057A00048176BEE7BE08CE297E00E94481764EEAE
:1057B0007BE082E397E00E94481783E090E09093BB
:1057C0006F0280936E0210926D0206CC84E190E02D
:1057D0009093B1028093B0024091670250916802A9
:1057E0006091690270916A028091630290916402F3
:1057F000A0916502B0916602481759076A077B07B6
:105800000CF076CFDB01CA0173CF85E190E0909375
:10581000B1028093B00288E893E1A0E0B0E068CFE5
:1058200087E090E09093A7028093A602109257021F
:10583000109258021092590210925A02E114F10487
:1058400099F0EA94EF2809F070CA87E190E090930C
:10585000B1028093B00280915F0290916002A091AA
:105860006102B091620244CF86E190E09093B10270
:105870008093B0028091670290916802A0916902C2
:10588000B0916A0235CF84E00E94370F882309F473
:105890004CCAA3E0CA1AD108B5E0CB16D10408F06F
:1058A00044CA1092B6020E9497129093B502809358
:1058B000B40282E090E0FECA81E00E94D9124FCA91
:1058C00080E00E94D91281114ACA88E00E94370FF5
:1058D000882309F444CA1092B6028091B0029091D4
:1058E000B1028D30910509F44EC060F50C9709F0B6
:1058F00036CA80915D0290915E02019690935E029D
:1059000080935D028091670290916802A091690284
:10591000B0916A0280599140A109B1098093670250
:1059200090936802A0936902B0936A0280915B022F
:1059300090915C02059790935C0280935B0282E0F9
:1059400090E041C08E309105E1F1419709F007CA1E
:105950008091670290916802A0916902B0916A02F9
:10596000885E9340A109B109809367029093680211
:10597000A0936902B0936A0282E390E0909371026F
:1059800080937002DCCF80915B0290915C020A965A
:1059900090935C0280935B02809167029091680211
:1059A000A0916902B0916A02885C9109A109B109CC
:1059B0008093670290936802A0936902B0936A0291
:1059C000BECF8FE090E09093B1028093B002C7C940
:1059D00084E00E94370F882309F440C01092B60279
:1059E0000E94F03022E030E040E050E00E94F332CC
:1059F000672B682B692BD9F46EE979E086E297E092
:105A00000E94481763E979E08CE297E00E9448170A
:105A100082E090E090936F0280936E0210926D028C
:105A20009093A7028093A6028BE090E0CCCF63E82E
:105A300079E086E297E00E9448176DE779E08CE212
:105A400097E00E94481782E090E090936F02809365
:105A50006E0210926D0289E090E0E2CF88E00E9431
:105A6000370F882309F47BC91092B60280915D023A
:105A700090915E02892BE9F46EE679E086E297E088
:105A80000E9448176FE579E08CE297E00E94481782
:105A900062E579E082E397E00E94481783E090E0B6
:105AA00090936F0280936E0210926D0288E090E0F6
:105AB000B7CF0E94F03022E030E040E050E00E949A
:105AC000F332672B682B692B49F461E579E086E2B4
:105AD00097E00E94481761E479E0B1CF80917202AB
:105AE000909173020197909373028093720218163B
:105AF00019064CF460E479E086E297E00E944817CA
:105B000060E379E09CCF0E94F03023EE34E040E087
:105B100050E00E94F3328B0102511D4F6EE179E09B
:105B200086E297E00E94481760E179E08CE297E016
:105B30000E944817B801872D962D0E940218672DE4
:105B4000762D8CE297E00E941717872D962D0E94E4
:105B500001156EEF78E082E397E00E9448176BEE44
:105B600078E088E397E00E94481784E090E0909303
:105B70006F0280936E0281E080936D02012E000C13
:105B8000220B330B8091670290916802A091690209
:105B9000B0916A02800F911FA21FB31F809367020A
:105BA00090936802A0936902B0936A02803B94408C
:105BB000A105B1051CF081E190E032CF82E090E0D8
:105BC0002FCF80E00E94D9128111C9C888E00E94BD
:105BD000370F882309F43FC18091B0029091B10240
:105BE0008431910509F4BDC098F48231910509F41E
:105BF0007FC04397F1F11092B6020E9497129093E2
:105C0000B5028093B4028091A6029091A702DBCEE8
:105C10008631910509F402C108F4CCC0479759F7C1
:105C200040915702509158026091590270915A0266
:105C300080915F0290916002A0916102B091620236
:105C4000841B950BA60BB70B80935F0290936002A9
:105C5000A0936102B0936202809167029091680202
:105C6000A0916902B0916A02840F951FA61FB71F09
:105C700036C080916B0290916C0220915702309156
:105C800058024091590250915A02880F991F880F6B
:105C9000991FFC01E457FD4FC080D180E280F38062
:105CA000C21AD30AE40AF50AC082D182E282F382E0
:105CB0008C589D4FDC016D917D918D919C910E943E
:105CC000FF340091670210916802209169023091BF
:105CD0006A02DC01CB01800F911FA21FB31F8093CA
:105CE000670290936802A0936902B0936A0283CF1F
:105CF00080916B0290916C02209157023091580272
:105D00004091590250915A02880F991F880F991F8C
:105D1000FC01E457FD4FC080D180E280F380C20EC9
:105D2000D31EE41EF51EC082D182E282F3828C581B
:105D30009D4FFC0160817181828193810E94FF34BB
:105D400000916702109168022091690230916A0205
:105D500068017901C61AD70AE80AF90AD701C6010B
:105D6000BECF4091570250915802609159027091F4
:105D70005A028091630290916402A0916502B091F1
:105D80006602841B950BA60BB70B8093630290935E
:105D90006402A0936502B0936602809167029091BD
:105DA0006802A0916902B0916A02841B950BA60B50
:105DB000B70B95CF4091570250915802609159020C
:105DC00070915A028091630290916402A0916502E1
:105DD000B0916602840F951FA61FB71F80936302C0
:105DE00090936402A0936502B0936602809167026B
:105DF00090916802A0916902B0916A02840F951F88
:105E0000A61FB71F8093670290936802A093690250
:105E1000B0936A0281E080935602EDCE4091570222
:105E2000509158026091590270915A0280915F021C
:105E300090916002A0916102B0916202840F951F5F
:105E4000A61FB71F80935F0290936002A093610228
:105E5000B0936202A2CF8FB7F8948090B80290906E
:105E6000B902A090BA02B090BB028FBF8091B0027D
:105E70009091B1024297C12CD12C7601C394029724
:105E800028F07AE0C72ED12CE12CF12C809152021F
:105E900090915302A0915402B09155029501840152
:105EA000081B190B2A0B3B0B809150029091510259
:105EB00044EF51E060E070E08230910554F044E638
:105EC00050E060E070E0853191051CF040E050E06A
:105ED000BA01401751076207730710F00C94AF2600
:105EE000843691050CF45CC05AE0252E312C412CEF
:105EF000512C8D379105BCF044E6242E312C412CD9
:105F0000512C863991057CF068EE262E63E0362E02
:105F1000412C512C8F3A910534F030E1232E37E299
:105F2000332E412C512C883E03E090072CF401962F
:105F300090935102809350020E942F0F87FF41C01F
:105F40008092520290925302A0925402B092550253
:105F500040914C0250914D0260914E0270914F025F
:105F60008091570290915802A0915902B0915A0223
:105F70008A019B010C191D092E093F0908171907F1
:105F80002A073B0794F08C0D9D1DAE1DBF1D80930D
:105F9000570290935802A0935902B0935A020DC031
:105FA000212C312C21012394C2CF409357025093CE
:105FB00058026093590270935A020E94B5140C94CF
:105FC000AF260E942F0F86FF39C080925202909216
:105FD0005302A0925402B0925502AAE0B0E0A70189
:105FE00096010E9412339B01AC01C201B1010E94D3
:105FF000FF340091570210915802209159023091BC
:106000005A02DC01CB01800F911FA21FB31F009128
:106010004C0210914D0220914E0230914F02081710
:1060200019072A073B070CF0B2CF009357021093D1
:1060300058022093590230935A02BFCF0E942F0F6B
:1060400084FF23C08092520290925302A092540285
:10605000B09255028091570290915802A091590236
:10606000B0915A028C159D05AE05BF052CF08C1918
:106070009D09AE09BF098BCF1092570210925802AA
:106080001092590210925A0298CF0E942F0F85FF4A
:106090002AC08092520290925302A0925402B0926F
:1060A0005502AAE0B0E0A70196010E9412339B01BD
:1060B000AC01C201B1010E94FF340091570210915E
:1060C00058022091590230915A02061717072807E3
:1060D000390794F268017901C61AD70AE80AF90A61
:1060E000D701C60154CF109252021092530210925F
:1060F00054021092550210925102109250020C94C8
:10610000AF26CF93DF938EE397E00E94011588E3DB
:1061100097E00E94011582E397E00E9401158CE24E
:1061200097E00E94011586E297E00E940115C8E6FB
:10613000D7E02697CE010E94011587E0C434D80726
:10614000C1F7DF91CF9108958F929F92AF92BF9246
:10615000CF92DF92EF92FF92CF93DF93EC016881B1
:1061600079818A819B81611571058105910521F4F1
:1061700064E279ED8BE597E02DE133EF41E050E00B
:106180000E94F33249015A019B01AC01A7EAB1E434
:106190000E9412336B017C01ACEEB4EFA5019401B7
:1061A0000E942033C60ED71EE81EF91EF7FE06C059
:1061B00081E0C81AD108E10880E8F80AC882D982CB
:1061C000EA82FB82C701B6019F77DF91CF91FF90F2
:1061D000EF90DF90CF90BF90AF909F908F900895F9
:1061E0008F929F92AF92BF92CF92DF92EF92FF92E7
:1061F000609115017091160180911701909118011D
:10620000611571058105910521F464E279ED8BE555
:1062100097E02DE133EF41E050E00E94F332490175
:106220005A019B01AC01A7EAB1E40E9412336B0151
:106230007C01ACEEB4EFA50194010E942033C60EA0
:10624000D71EE81EF91EF7FE06C081E0C81AD10865
:10625000E10880E8F80AC0921501D0921601E09298
:106260001701F0921801C701B6019F77FF90EF90D8
:10627000DF90CF90BF90AF909F908F9008956093E4
:1062800015017093160180931701909318010895DA
:10629000FB01DC0105900D920020E1F70895FC015F
:1062A00005900020E9F7809590958E0F9F1F089527
:1062B000BB274A3031F4992322F4BDE290958195B1
:1062C0009F4F0C949531BB272A3051F4992342F407
:1062D000BDE290958095709561957F4F8F4F9F4F50
:1062E0000C947331BB27FA01A62F62177105810543
:1062F0009105330B30FB66F0AA27660F771F881FC6
:10630000991FAA1FA21710F0A21B63953850A9F776
:10631000A05DAA3308F0A95DA19336F7B111B1933E
:106320001082CA010C94AE31BB27FB015527AA2766
:10633000880F991FAA1FA41710F0A41B8395505112
:10634000B9F7A05DAA3308F0A95DA193009779F78A
:10635000B111B1931192CB010C94AE31DC01FC016F
:10636000672F71917723E1F7329704C07C916D9389
:1063700070836291AE17BF07C8F30895E89409C00F
:1063800097FB3EF490958095709561957F4F8F4F68
:106390009F4F9923A9F0F92F96E9BB279395F6957E
:1063A000879577956795B795F111F8CFFAF4BB0FFC
:1063B00011F460FF1BC06F5F7F4F8F4F9F4F16C060
:1063C000882311F096E911C0772321F09EE8872FEA
:1063D000762F05C0662371F096E8862F70E060E0A6
:1063E0002AF09A95660F771F881FDAF7880F96951F
:1063F000879597F90895990F0008550FAA0BE0E8C3
:10640000FEEF16161706E807F907C0F01216130676
:10641000E407F50798F0621B730B840B950B39F4B6
:106420000A2661F0232B242B252B21F408950A261C
:1064300009F4A140A6958FEF811D811D08950E944A
:1064400032320C94A3320E94953238F00E949C3272
:1064500020F0952311F00C948C320C94923211247C
:106460000C94D7320E94B43270F3959FC1F3950F0C
:1064700050E0551F629FF001729FBB27F00DB11DC8
:10648000639FAA27F00DB11DAA1F649F6627B00D58
:10649000A11D661F829F2227B00DA11D621F739F41
:1064A000B00DA11D621F839FA00D611D221F749F4F
:1064B0003327A00D611D231F849F600D211D822F96
:1064C000762F6A2F11249F5750409AF0F1F08823BD
:1064D0004AF0EE0FFF1FBB1F661F771F881F9150EA
:1064E0005040A9F79E3F510580F00C948C320C94DB
:1064F000D7325F3FE4F3983ED4F38695779567955E
:10650000B795F795E7959F5FC1F7FE2B880F911D13
:106510009695879597F9089597F99F6780E870E0B9
:1065200060E008959FEF80EC089500240A94161609
:10653000170618060906089500240A941216130671
:10654000140605060895092E0394000C11F48823FF
:1065500052F0BB0F40F4BF2B11F460FF04C06F5F1B
:106560007F4F8F4F9F4F089557FD9058440F551FF1
:1065700059F05F3F71F04795880F97FB991F61F0C5
:106580009F3F79F087950895121613061406551F3C
:10659000F2CF4695F1DF08C0161617061806991FA8
:1065A000F1CF86957105610508940895E894BB279D
:1065B00066277727CB0197F90895F999FECF92BD09
:1065C00081BDF89A992780B50895262FF999FECFB5
:1065D0001FBA92BD81BD20BD0FB6F894FA9AF99A00
:1065E0000FBE01960895052E97FB1EF400940E949D
:1065F0000A3357FD07D00E945C3307FC03D04EF4EA
:106600000C940A3350954095309521953F4F4F4F4C
:106610005F4F089590958095709561957F4F8F4F4E
:106620009F4F08950E947E33A59F900DB49F900DBB
:10663000A49F800D911D11240895B7FF0C9412336F
:106640000E941233821B930B08952F923F924F9218
:106650005F926F927F928F929F92AF92BF92CF92F2
:10666000DF92EF92FF920F931F93CF93DF93CDB7FB
:10667000DEB7CA1BDB0B0FB6F894DEBF0FBECDBF73
:1066800009942A88398848885F846E847D848C8444
:106690009B84AA84B984C884DF80EE80FD800C814D
:1066A0001B81AA81B981CE0FD11D0FB6F894DEBF30
:1066B0000FBECDBFED010895A1E21A2EAA1BBB1B90
:1066C000FD010DC0AA1FBB1FEE1FFF1FA217B307BE
:1066D000E407F50720F0A21BB30BE40BF50B661FD4
:1066E000771F881F991F1A9469F760957095809598
:1066F00090959B01AC01BD01CF010895A29FB0010F
:10670000B39FC001A39F700D811D1124911DB29FE5
:10671000700D811D1124911D08955058BB27AA2783
:106720000E94A5330C94A3320E94953238F00E9447
:106730009C3220F039F49F3F19F426F40C949232E5
:106740000EF4E095E7FB0C948C32E92F0E94B432F2
:1067500058F3BA17620773078407950720F079F496
:10676000A6F50C94D6320EF4E0950B2EBA2FA02D80
:106770000B01B90190010C01CA01A0011124FF27EE
:10678000591B99F0593F50F4503E68F11A16F040E9
:10679000A22F232F342F4427585FF3CF46953795E8
:1067A0002795A795F0405395C9F77EF41F16BA0BAD
:1067B000620B730B840BBAF09150A1F0FF0FBB1F5B
:1067C000661F771F881FC2F70EC0BA0F621F731FA4
:1067D000841F48F4879577956795B795F7959E3F01
:1067E00008F0B0CF9395880F08F09927EE0F979592
:1067F000879508950E940E340C94A3320E949C3217
:1068000058F00E94953240F029F45F3F29F00C9433
:106810008C3251110C94D7320C9492320E94B432C3
:1068200068F39923B1F3552391F3951B550BBB27BF
:10683000AA2762177307840738F09F5F5F4F220F04
:10684000331F441FAA1FA9F335D00E2E3AF0E0E8FB
:1068500032D091505040E695001CCAF72BD0FE2F45
:1068600029D0660F771F881FBB1F261737074807D9
:10687000AB07B0E809F0BB0B802DBF01FF27935891
:106880005F4F3AF09E3F510578F00C948C320C9497
:10689000D7325F3FE4F3983ED4F3869577956795BA
:1068A000B795F7959F5FC9F7880F911D96958795C6
:1068B00097F90895E1E0660F771F881FBB1F6217E5
:1068C00073078407BA0720F0621B730B840BBA0BA3
:1068D000EE1F88F7E09508950E9473346894B11113
:1068E0000C94D73208950E94BC3288F09F5798F0DC
:1068F000B92F9927B751B0F0E1F0660F771F881FC5
:10690000991F1AF0BA95C9F714C0B13091F00E94DE
:10691000D632B1E008950C94D632672F782F8827AD
:10692000B85F39F0B93FCCF3869577956795B39505
:10693000D9F73EF490958095709561957F4F8F4F74
:106940009F4F08950E94E23490F09F3748F49111D0
:1069500016F00C94D73260E070E080E89FEB089569
:1069600026F41B16611D711D811D0C94B9340C9405
:10697000D434882371F4772321F09850872B762F15
:1069800007C0662311F499270DC09051862B70E043
:1069900060E02AF09A95660F771F881FDAF7880F54
:1069A0009695879597F908959F3F31F0915020F47F
:1069B000879577956795B795880F911D96958795DB
:1069C00097F908950E94BC32A0F0BEE7B91788F489
:1069D000BB279F3860F41616B11D672F782F8827C4
:1069E000985FF7CF869577956795B11D9395963902
:1069F000C8F308950E94FB3108F48FEF0895DB017E
:106A00008F939F930E941233BF91AF91A29F800DED
:106A1000911DA39F900DB29F900D11240895EE0F2C
:106A2000FF1F0590F491E02D09940F931F93CF93CE
:106A3000DF938230910510F482E090E0E0918207CC
:106A4000F091830730E020E0B0E0A0E0309799F4C7
:106A50002115310509F44AC0281B390B24303105B2
:106A6000D8F58A819B816115710589F1FB019383BA
:106A70008283FE0111C04081518102811381481738
:106A80005907E0F04817590799F4109761F01296EA
:106A90000C93129713961C933296CF01DF91CF91EE
:106AA0001F910F9108950093820710938307F4CFED
:106AB0002115310551F04217530738F0A901DB01C8
:106AC0009A01BD01DF01F801C1CFEF01F9CF909329
:106AD000830780938207CDCFFE01E20FF31F8193DE
:106AE00091932250310939832883D7CF2091800791
:106AF00030918107232B41F420911B0130911C011F
:106B000030938107209380072091190130911A0159
:106B10002115310541F42DB73EB740911D0150912B
:106B20001E01241B350BE0918007F0918107E217CD
:106B3000F307A0F42E1B3F0B2817390778F0AC01A0
:106B40004E5F5F4F2417350748F04E0F5F1F50937D
:106B5000810740938007819391939FCFF0E0E0E01D
:106B60009CCFCF93DF930097E9F0FC01329713821B
:106B70001282A0918207B0918307ED0130E020E0FE
:106B80001097A1F420813181820F931F20918007FB
:106B9000309181072817390709F061C0F093810708
:106BA000E0938007DF91CF910895EA01CE17DF07C8
:106BB000E8F54A815B819E0141155105B1F7E90174
:106BC000FB83EA8349915991C40FD51FEC17FD0748
:106BD00061F4808191810296840F951FE901998368
:106BE0008883828193819B838A83F0E0E0E0129620
:106BF0008D919C9113970097B9F52D913C91119728
:106C0000CD010296820F931F20918007309181075A
:106C10002817390739F6309751F5109283071092EB
:106C20008207B0938107A0938007BCCFD383C28330
:106C300040815181840F951FC817D90761F44E5FB9
:106C40005F4F88819981480F591F518340838A8102
:106C50009B81938382832115310509F0B0CFF09396
:106C60008307E09382079ECFFD01DC01C0CF138232
:106C70001282D7CFB0E0A0E0E0E4F6E30C94273333
:106C80008C01009751F4CB010E9415358C01C8018D
:106C9000CDB7DEB7E0E10C944333FC01E60FF71FFC
:106CA0009C0122503109E217F30708F49DC0D90175
:106CB000CD91DC911197C617D70798F0C530D10553
:106CC00030F3CE0104978617970708F3C61BD70B3E
:106CD0002297C193D1936D937C93CF010E94B135DC
:106CE000D6CF5B01AC1ABD0A4C018C0E9D1EA09143
:106CF0008207B0918307512C412CF12CE12C109785
:106D000031F580918007909181078815990509F0E8
:106D10005CC04616570608F058C080911901909142
:106D20001A01009741F48DB79EB740911D01509113
:106D30001E01841B950BE817F90708F055C0F09366
:106D40008107E0938007F90171836083A0CF8D9163
:106D50009C91119712966C90129713967C901397B2
:106D6000A815B90559F56C0142E0C40ED11CCA142E
:106D7000DB0420F1AC014A195B09DA011296159780
:106D800080F06282738251834083D9016D937C933A
:106D9000E114F10471F0D7011396FC93EE9312976E
:106DA00076CF22968C0F9D1FF90191838083F3018A
:106DB000EFCFF0938307E093820769CF4816590617
:106DC00008F42C017D01D3019ACFCB010E94153527
:106DD0007C01009749F0AE01B8010E94F736C80166
:106DE0000E94B135870153CF10E000E050CFFB0186
:106DF000DC0102C001900D9241505040D8F7089537
:106E0000FB01DC018D91019080190110D9F3990BE0
:106E10000895FB01DC0101900D920020E1F7089537
:106E200017E0CFEDD7E004C0FE010E940F35219698
:0A6E3000C03ED107C9F7F894FFCF68
:106E3A0010400D0300A0860100FFFFFFFF00E100E4
:106E4A00000000000001000000000084078000002C
:106E5A00C1808100000000000000280C930D490C3D
:106E6A003E0C8F0C4D0C6B0C000000003312FD0E13
:106E7A00A813180E00000000E511FD0EA813180E45
:106E8A0000000000AD10FD0EA813180E596F7520F2
:106E9A006F776E2000736C6E6700596F752065619D
:106EAA007420697420616C6C2062757400666F725C
:106EBA0067657420746F20627275736820796F75C4
:106ECA00720074656574682E205468657920616C57
:106EDA006C20726F7400616E6420796F7520636133
:106EEA006E27742065617400736F6C696420666F25
:106EFA006F6420616E796D6F72652E002020204AC2
:106F0A0075737420736179206E6F002020202074BD
:106F1A006F2063616E64792E00696E2061206C7542
:106F2A006E636820626F7820696E007468652073EA
:106F3A00756277617921212100546865206D61723B
:106F4A006B657420686173006265656E20666C6F9C
:106F5A006F6465642077697468006368656170208E
:106F6A00686F6D656D616465004165726F212121ED
:026F7A002100F4
:00000001FF
